:020000041100E9
:103000000023F7B52E4D2F4C280063616374022610
:1030100001F070F94021FE22217428002A4B00960D
:1030200001F0BAF900283AD1217CFF222800274B71
:10303000009601F0B1F9002831D1254BA2899A42BE
:103040002AD1E389234A934211D1234B6361234B55
:103050002268002A07D1002B05D019002200C1C91F
:10306000C1C21B7B6374280001F082F9F7BD1C4AC2
:10307000934201D00023EBE71A4B1B4A1B68934293
:1030800006D9C02304222800217C9B0001F0FAF914
:10309000164B6361164BDBE700232374EAE7CC236E
:1030A0003821AC2228009B01217401F0EBF90028A3
:1030B000F2D1104B6361104BE381104BC8E7C0465F
:1030C000D441FF1FA061FF1FAC61FF1FAE61FF1F56
:1030D00059590000830500002541001140BD001131
:1030E00082150000C461FF1F87130000D941001141
:1030F00050BD001171410011AAAAFFFF30BD00119F
:10310000F7B5164B0192C318021D002000938823C7
:103110005B05D3181B685C1C1AD09CB2402C18D8D5
:103120008D781E0CAC466746CD782D023D43AE42ED
:1031300006D1019800280ED110000C70240A4C70A2
:1031400003249BB20733A343D218009B9A42DED3D9
:10315000FEBD4432F9E71000FAE7C046FC0F00005C
:10316000802213B503000324019189B25201073173
:103170009B18A14304305A1A88235B05C3181B68A7
:10318000591C03D190429241104016BD99B240297A
:1031900007D80B000733A343C0189042ECD300209C
:1031A000F3E74430F9E7134B134A1B68126810B574
:1031B000FA24934201D81A00F824104BE4021B6849
:1031C0009A4210D813000E4A12689A420ED3013365
:1031D00007D1F823DB029C4203D10A49054808F0D5
:1031E00043FB200010BDFC24E402ECE7FE24E402D3
:1031F000F7E7C04600C0071100D0071100E0071133
:1032000000F00711FFFFFF7FF0B59BB015000490A1
:103210000391402A00D9A0E006AB59801A80FFF73D
:10322000C2FF0400042816D9002206A9FFF768FF90
:10323000052810D906AB1B88AB420CD1002D07D056
:10324000514B2A000499C01808F0DEFA002802D178
:1032500001201BB0F0BD06AB1D8020000699FFF7D2
:103260007FFF041E7BD1069B0793FFF79CFF802303
:103270005B01C618802307001B039E4201D3F8267A
:10328000F60288235B05F31801931B68013302D013
:10329000019808F029FB3D49019808F0E5FA3B1D2B
:1032A0000293331D05938822029B52059B181B68CD
:1032B00008935A1C3CD044219AB20091402A04D869
:1032C0000320D11D814389B2009103991B0C8B42CD
:1032D00024D0402A22D80122300008A9FFF710FF8D
:1032E000021E1BD1380008A9FFF70AFF04000428BA
:1032F00031D9009A059B9B1880225201B218934243
:1033000040D288235B05C118009A09A808F054FA36
:103310001D4B009A09A9F01808F0D6FA009A029BF2
:103320009446634402931A4B029AFB189A42BAD30A
:1033300088235B05FC1821680198013908F094FA8C
:10334000200008F0D1FA039A07AB5A8030000799A1
:10335000FFF706FF0400002C03D1002079E70428C2
:10336000FBD988235B05E018069908F07DFA032352
:10337000EA1C9A4300D16BE7034B0499E01808F06C
:10338000A3FA65E70424ECE704000011FFFFFF7FC8
:10339000F80F0000F7B505001400402A21D80027D7
:1033A00001AE71803780FFF7FEFE042816D93A007F
:1033B0003100FFF7A5FE042810D93688BC420BD097
:1033C000BD4209D0221CB44200D9321C064B92B235
:1033D000C118280008F0F0F930B2FEBDC04300B2B9
:1033E000FBE703204042F8E70400001137B5042250
:1033F00004000D0001A81649FFF7CCFF02000428C5
:103400000BD1019BA34208D3AB4204D0104901A8C1
:103410000195FFF7F9FE01203EBD0E4C2368200008
:10342000019308F061FA019920000139019108F037
:103430001BFA80235B01E418074B9C42EED1042267
:10344000034901A80195FFF7DFFE0020E4E7C0462D
:103450005555000000C007110000081130B589B0B3
:1034600008F0F2F910226946254808F015FB254BB3
:10347000009A9A420ED1019B029A0F2B33D8002159
:1034800001240698013B08D2002900D00292029B39
:10349000013331D10023029325E0551CF2D1020003
:1034A0002100EFE710341022200004A908F0F4FAFC
:1034B000029B013301D1069B0293882304995B058B
:1034C000C918059B06981A03120B049105928142B4
:1034D00003D02B4201D108F06FF9019B013B01930E
:1034E000019B002BDED1029B002B03D00493049898
:1034F0004168084709B030BDE025014C2D03EFE7D6
:1035000000000111504859368022F8B5964C974B6F
:10351000D200002120001C6008F05EFB2300944ACA
:1035200088331A60934B1A786A23002A00D011332B
:10353000E3620A232365904B37221B780820A3639C
:103540008E4B2118E361102323628D4B3B25636171
:10355000C823DB00A36123008C331A602823013ABF
:10356000E26320646364CA67043A211DCA672100CC
:10357000BC310D602100C03108602100C4310B60F6
:1035800021000635CC310D602100083DC8310D60A9
:103590002100D0310A602200D43210602200D832DB
:1035A000136022000227E032210017604222DC3142
:1035B0000A6021001B3DE4310D602100E831086004
:1035C0002100EC310B6023000521F4331960230046
:1035D000F0331A602300183290331A6023009433BA
:1035E000186023001E3A98331A60AF23DB00236073
:1035F000644BFA262363644B644DE360644BF03103
:10360000A3642300FF31FC33B600A16021611E607A
:10361000A5627325E5656D3D6565A56596255D4AE1
:10362000AD00E264666258606766A56600270925FA
:10363000A767E566584F594D606720002567E26728
:103640003A6015279C30676007001A203860200018
:10365000A0300700212038602000A83007004C4827
:1036600038602000F830066026006427A4363760F2
:1036700026005F3FAC3637602600033FB036376028
:103680002600C637B436376026000027B8363760C4
:1036900038269E60424E96205E64424E5A66DE6137
:1036A000414E9A645E62F53EFF3E9E621E269A6718
:1036B000354A8000DE661F675F67DD651D6618623C
:1036C000DA67BE23394A5B00E250394BD8382350C1
:1036D00004302250C4225200A350C623E4205B00D1
:1036E000E1500433334AE1503349344BD16034491B
:1036F000800019503349E938FF38195032490430F5
:10370000195032493248D16132491163324951630B
:103710001900F4310860CE20304940001160304972
:10372000195019002F48F83108602F49D1658221BE
:103730002E4A89005A501A002D490832D1671A00C2
:103740002C49B432116088212B4A89005A501A0042
:103750002A49883211602A4ADA6408F0BDF801204B
:1037600007F0EAFFF8BDC0460004FF1F4464FF1FD6
:10377000106FFF1F1044FF1F4A0AFF1F3A07000087
:1037800080C3C9019A020000DC0500006A1800002D
:1037900050C3000088130000F009FF1F204E0000F6
:1037A0006509FF1F68100000C409000040420F00B7
:1037B00010270000FC00FF1F791CFF1F0000FF1FE7
:1037C000CD2CFF1F5530FF1FED2EFF1F3920FF1F8F
:1037D0002927FF1F5520FF1F0122FF1FC51FFF1FA5
:1037E0004D29FF1F352AFF1F9119FF1F5928FF1F61
:1037F0007D25FF1F8925FF1FC51EFF1F7D1FFF1F82
:103800003D1EFF1F0223F0B50124604D604E2B705A
:10381000604B91B01C70604F03933368002120000F
:10382000FB7006F0FFFD200006F0F6FC0023984236
:1038300005D0FA78552A02D0332A00D099E03360B7
:10384000042006F057FF07F0D7FEFFF75DFE08F0F3
:10385000EBF81F2201240021504B10AE1A70504B80
:103860001C70504B1970504B19689143163A0A431B
:103870001A60602219689143403A0A431A6008F0BE
:10388000CBF908F0F9F8494B9847C120FF21484B84
:1038900080001A588A431A50C522920098588843CB
:1038A000BF39014399509858424908408021C901C5
:1038B0000143802099509958C0050902090A014323
:1038C000995080213C48490108F05EF8032322000A
:1038D0003A49019400933A4807F0E6FF2C2239490F
:1038E00005A807F069FF05AC61782078023406F07E
:1038F000B3FCA642F8D1344C344B226803201A4062
:10390000A023DB0213432360802322689B0413431C
:10391000236022682E4B1A4080239B0313432360AD
:103920002C4A2D4B934200D8012008F0C5F808F02E
:103930005BF980232268DB0413432360287808F0B6
:10394000FBF8039B1878C0B208F046F808F054F86A
:103950002249042008F0D0F806F098FE00F040F864
:1039600000F0E6FD00F08EFE00F00AFA002011B033
:10397000F0BD00932100194A042008F0CDF88023FF
:10398000DB059C62FFF76AFD5AE7C0464A0AFF1F43
:1039900034F000401044FF1FD061FF1F480AFF1F92
:1039A000490AFF1F680AFF1FBCF00040E1A20000A7
:1039B00000E100E0FF00FFFF1444FF1F9856FF1FC7
:1039C0001454FF1F58BC001114F00040FF7FF8FF93
:1039D000FFFF9FFF0080FF1F106FFF1F3B000108CC
:1039E000002210B51100112007F016FE10BD0000D6
:1039F000F8B500230926364F364C3B62E3681120A8
:103A0000B343E36007F0E8FE112008F09DF81120B1
:103A100007F0A2FE40232268102513432360802371
:103A20006268DB02134363608023A26802211343B0
:103A3000A360A368284A08201340A3608023A268DB
:103A40009B0113430122A360236CAB432364236CCB
:103A50001343236480231B013B62226B1F4B1A40DC
:103A60002263626B1A406263A26B1A40A263E26B2C
:103A70001340E363E3681A4A1340E36006F0ECFB8B
:103A80000121082006F0FCFC8023164A5B00516CE3
:103A900011200B43536407F047FFFD21C720124B51
:103AA000124A89005A50A36B80002B43A363E3683A
:103AB0000F4A3343E3600F4B195811408022120222
:103AC0000A431A50802292051A600B4B5D63F8BDC1
:103AD00000F000403CF00040FFFFDFFFEFFFEFFF92
:103AE000FFFF7FFF003800400000FF1F5118FF1F3D
:103AF000FF00FFFF00E100E00000054070B5284C2A
:103B0000238C002B23D0228A002A21D1DA002382A1
:103B10006382A382E38223836383A383E38322609C
:103B20006260A260E2601F4D1F4A6420EB809342F6
:103B30000AD8FA220020D200934205D91B4A0A2152
:103B4000981807F011FFC0B200232872238470BDBB
:103B50000720E11CCA7F01320240CA7705D1032544
:103B6000201DC17F01312940C17708325200A35284
:103B7000002321001A00088A01321B180231082A8A
:103B8000F9D1221DD27F9200A350626823689B184E
:103B9000A2689B18E2689B185B099BB2C3E7C0460A
:103BA0001061FF1FB861FF1FB70B000030F8FFFF67
:103BB00030B503A804880B20002C0ED14968074DAE
:103BC00008784978090201430A20A94205D1012158
:103BD00020001980024B1B7A137030BD192A000097
:103BE000B861FF1FF7B5150008AA16884A680F4F7D
:103BF00014785278120222430A24BA4214D10122C4
:103C0000DBB2019200962A0007F090FC041E0BD153
:103C1000074B1B68002B07D068782A7800021043F6
:103C200042425041013098472000FEBD0229000069
:103C30003C61FF1F30B5012503790400BFB02B4262
:103C400011D00A49408806F0DDFF28420BD0084B0E
:103C500001A95B8D4D800B80064B00221B7A60888A
:103C60000B7104F0C1F83FB030BDC0463461FF1F96
:103C70004840FF1FB861FF1F10B50549054806F011
:103C800077FF0421044A054806F034FF10BDC04602
:103C90003461FF1FFFFF000084BC00114840FF1F7C
:103CA00010B5024804F022FF10BDC046353C00119B
:103CB000012303700B4B1A7A4270022282709A78A9
:103CC000C270DA780271032242711A7982715A79CC
:103CD000C2710C2202729A794272DB7983720B20D4
:103CE0007047C046B861FF1F022310B50370013B47
:103CF00043700533837010330371443B43712A339F
:103D000083714433C37100230372064B04001B8884
:103D100043720A30FFF7CCFF831D0A30C0B2E37054
:103D200010BDC046B861FF1F10B5142007F0C4FCD9
:103D3000124B14220021186007F04EFF002007F0FC
:103D400023FF012007F0B8FD022007F035FE032015
:103D500004F070F9042006F085F9052003F0AEFBAD
:103D6000062004F07BF8072001F060FA082006F036
:103D7000A1FE092001F03AF810BDC0464061FF1FC6
:103D800007F0AAFC012007F05FFC07F0ADFC000083
:103D9000094B10B50400984205D0012904D1200038
:103DA000064906F0E5FE10BD0229FCD1013904F0F8
:103DB0005BFE0028F3D0F6E7FEFF00006661FF1F00
:103DC00070B50D7A100004AA2C0016881022144039
:103DD000154220D1002E20D10A78022A18D14A6833
:103DE000517815780E4A09022943914205D00D4AAF
:103DF000914209D01C800A2404E014220A491A8046
:103E000007F0DAFC200070BD0C2208491A80F7E7A1
:103E10001C800124F6E70824F4E70B24F2E7C046EF
:103E2000F3FF0000F4FF00009C42FF1F6CBD001177
:103E300010B504000749084806F09AFE074804F048
:103E400095FD0020E40704D50721054A054806F042
:103E500051FE10BD6661FF1FFFFF0000913D001184
:103E6000C8BC00118C40FF1F00B50C4BBFB01A78C6
:103E70000B4902A800F0C0FC6B4680B2D880002835
:103E800009D06A46074B01A91B889380064B002284
:103E9000188803F0A9FF3FB000BDC0464461FF1F72
:103EA0004561FF1FE640FF1FF041FF1F00B50C4BAF
:103EB000BFB01A780B4902A801F0DCFE6B4680B255
:103EC000D880002809D06A46074B01A95B8D9380F2
:103ED000064B0022188803F087FF3FB000BDC046A4
:103EE0006E61FF1F6F61FF1F8C40FF1FF041FF1FBE
:103EF000F7B50E00377A1C0008AB11003D001A8898
:103F000020231D401F423CD13378022B3BD17368E4
:103F10001F785B781B023B431E4FBB4208D01E4FED
:103F2000BB4214D01D4DAB4221D00A252800FEBD56
:103F3000002A2AD1142C2AD82200F06807F03CFC71
:103F4000174B1C70012CF1D9FFF7B0FFEEE7002AE8
:103F50001BD1202C1BD82200F06807F02DFC114B40
:103F600004211C70104B187807F07EFDDEE7E3B2E9
:103F70000124009201940A00310007F0D7FA0500ED
:103F8000D4E70825D2E70125D0E70B25CEE70D259C
:103F9000CCE7C046F3FF0000F4FF00000229000058
:103FA0006E61FF1F4461FF1FF061FF1F332310B5D7
:103FB000040003700A220749013007F0FDFB064B9D
:103FC0000F201B681A0AE37222731A0C1B0E62730D
:103FD000A37310BDB861FF1FE061FF1F30B501255D
:103FE00003790400BFB02B4213D00B49408806F080
:103FF00009FE28420DD06A46084B02A81B88938010
:10400000FFF7D4FF6B46D8800022608801A903F037
:10401000EBFE3FB030BDC0466661FF1FE640FF1FAC
:1040200010B5024804F062FD10BDC046DD3F00112E
:1040300070B5160004AA148805AA15784A68507845
:10404000117800022A4A0843801805284BD807F047
:10405000A3FD03131E29343F0720032C0BD8042291
:10406000121BAA4200D92A0022491A8030000919DD
:1040700007F0A2FB002070BD0720112CFBD81222F4
:10408000121BAA4200D92A001B491A80EEE707201A
:104090000E2CF0D80F22121BAA4200D92A00174971
:1040A0001A80E3E70720032CE5D80422121BAA425A
:1040B00000D92A0012491A80D8E70720032CDAD841
:1040C0000422121BAA4200D92A000E491A80CDE709
:1040D0000720032CCFD80422121BAA4200D92A00A1
:1040E00009491A80C2E700220A201A80C3E7C046A5
:1040F000DCD5FFFF13BD00118C61FF1F03BD001154
:10410000FEBC0011F9BC0011F4BC001110B50D216A
:10411000024A034806F0EEFC10BDC046E8BC0011A0
:10412000FC40FF1F13B5104C0423217C01AA00F0B2
:1041300061F9002815D16B469A88236852BA92B269
:104140005343228909491B0C9B184B806B46DA8824
:10415000636852BA92B2534362891B0C9B188B80DE
:1041600016BD0120FCE7C046A061FF1FB861FF1F1C
:1041700037B5174C07236A46217C00F03BF900282D
:1041800024D16B461B787F2B20D86B46DD78F0233B
:104190002A041B031A406B469B880E495BBA9BB2EC
:1041A0001A4323682D09534322891B0C9B184B800B
:1041B0006B465A789B7812031B011A4363682A43A3
:1041C000534362891B0C9B188B803EBD0120FCE78A
:1041D000A061FF1FB861FF1F7FB50226154C0022AA
:1041E000217C03AB0096050000F0D6F8002802D031
:1041F000012004B070BD0E23217C0122280000960E
:104200006B4400F0C9F80028F2D16B469A89236804
:10421000D2BA5343228908491B149B184B806B4622
:10422000DA89636852BA92B2534362891B0C9B18B5
:104230008B80DEE7A061FF1FB861FF1F70B5114CD6
:10424000237C002B0FD0382B0ED10F4D280000F00F
:1042500051F8CC23AC222800217C9B0100F012F9FC
:10426000280000F085F870BD084BE2899A42FAD127
:10427000054D280000F03EF800222800217C00F0C7
:10428000E3F8EDE7A061FF1FD441FF1F83050000A5
:1042900070B5144C237C002B1FD06369002B1CD0FD
:1042A000114D280000F026F86369280098470400A3
:1042B000280000F05DF8002C10D10C4B0422995E10
:1042C000002905DA9C801A8801321A80200070BD0E
:1042D000074A9142F7DD9A80F5E70124FEF790FE48
:1042E000F4E7C046A061FF1FD441FF1FB861FF1F64
:1042F0000F27000070B5C17905000C00631E9C41BA
:104300001A4BE402E41849000460C9B2007906F0CF
:10431000EDF8E979687949000131C9B206F0E6F8AB
:10432000E8790930C0B207F017FA0023E366613379
:104330002360AA795B3B002A0ED022689A43023B95
:10434000134323600A23E3610733236200232363BB
:10435000A3630133E36370BD22689A4302231343CE
:104360002360462363610633A361EFE700500040FA
:1043700070B5002504000368DD66C0790930C0B25D
:1043800007F02AFA2900207906F04CF82900607914
:1043900006F048F870BD0000F8B51E0006AB1D78A9
:1043A000002304681700E366616007F04DFA0123FB
:1043B0008022E3662B0027615200013B08D207F000
:1043C000C3FA08200A4A1168002D03D12800F8BD5D
:1043D0002261F2E7236F034203D02369013D33706A
:1043E000013613685B1A032BEED90125EEE7C046B0
:1043F0006008FF1F70B51C00002305681600EB66FF
:10440000696007F021FA01238022EB662300520045
:10441000013B08D207F098FA08200A4A1168002CDC
:1044200003D1200070BD2A61F2E72B6F034203D055
:104430002B69013C3370013613685B1A032BEED9EC
:104440000124EEE76008FF1F002370B50468150023
:10445000E366616007F0F8F90123E366256107F080
:1044600073FA8020064A80001168636B034205D10D
:1044700013685B1A032BF8D9012070BD0020FCE7FC
:104480006008FF1F70B51D00002304681600E36676
:10449000616007F0D9F90123E36626610F33626B8F
:1044A0001A42FCD02B0A23611023626B1A42FCD003
:1044B000EDB2256107F048FA8020074A80001168B4
:1044C000636B034205D113685B1A032BF8D90120F3
:1044D00070BD0020FCE7C0466008FF1F70B51E00DD
:1044E000002305681400EB66696007F0ADF901234D
:1044F000A619EB660F33B4420ED107F025FA8020DF
:104500000A4A800011686B6B03420CD113685B1A76
:10451000032BF8D9012070BD21782961696B1942FC
:10452000FCD00134E7E70020F5E7C0466008FF1F34
:1045300010B5084CE368002B08D18022064B5202CC
:104540001B689B186360054B1B68236007F06CF8C1
:10455000A06010BDE061FF1FC8F00040CCF000403B
:1045600070B5184A936A916A9942FBD116498A68D4
:104570009A421FD39A1A8B60144B0126186893B283
:10458000D202D20E4343424300204C681B0A1B193F
:1045900012029B180E4C0A684B60551CA3420CD8A3
:1045A000002801D04B600A600A4A136008680A4B71
:1045B000186070BD581E821ADDE7084A30009B184B
:1045C0002A00EAE700F00040E061FF1F140AFF1F25
:1045D00040420F00C8F00040CCF00040C0BDF0FFEA
:1045E00070B51F4C23793F2B01D93F2323711D4BFD
:1045F00022791A701878C0B207F016FB18231A49EE
:104600001A4A0B801A4913800B805380A3791949E9
:1046100080200B800C21938001334B43164D191CD5
:104620000001834200D9011C2980D1806379002BCD
:1046300011D101336371237A012B01D80223237234
:104640006279237A0D4853430A21584307F08CF9C5
:104650000B4D286070BDA02BEDD9A023EAE7C04622
:10466000D461FF1F480AFF1FEE41FF1FBC43FF1F1D
:10467000EC41FF1FEA41FF1FE841FF1F71020000EC
:10468000C461FF1FF8B518210020FEF7AFFE114CE2
:10469000011E114D09D10C22104BC1CBC1C4280001
:1046A00007F09AFAFFF79CFFF8BD0C2220000C4996
:1046B000FEF770FE0C2802D0084B43CB43C40C22FB
:1046C00028000849FEF766FE0C28EBD00C220021DA
:1046D000E5E7C046D461FF1FA061FF1F60BD001168
:1046E000FC0C0000F50C0000F0B51D4C8022A54428
:1046F0000400882069465201400507F01DF9902208
:1047000012016A441300200032C832C316C816C30F
:104710008023144C144FA6689B033343A3603B6073
:1047200007F0B2F98823A0685B05C01807F0DCF831
:104730000025882329008022A0685B05C018401945
:104740006944520007F0C0F880230135FF355B0152
:104750009D42EED1A6603E60044B9D44F0BDC04634
:10476000FCEFFFFF2C43FF1F9808FF1F0410000001
:10477000F0B5040087B0002825D0684606F05CFF3D
:104780001B4C022806D106226946200007F03CF89F
:10479000002816D06946002301250F262F00E25C71
:1047A000013310091030874038002F003240974005
:1047B0003A0002434A610439062BEFD16846FFF7FD
:1047C00093FF07B0F0BD182269460A4807F0B4F815
:1047D0006A46A300D358013305D01822FF2168464A
:1047E00007F0FAF9EAE70134062CF1D1E9E7C0460F
:1047F0006509FF1F00090011F0B5002504000E0037
:1048000085B0AA4200D186E04B1C087801934B7812
:104810008978377909021943F3783F061B040B4363
:104820001F43039720706570252800D196E033D888
:10483000112813D807F008F969002B012B012B016F
:104840002B01AA00B800B1002B012B012B012B0179
:104850002B012B012B012B0105012501232800D160
:10486000DEE0DB2800D034E1042A00D8ACE01025DB
:10487000052A05D0551F2A003800711D06F09CFF3F
:1048800005223100200006F097FF2A003900601D44
:1048900006F092FF05353EE0562859D010D833284F
:1048A00000D19DE0552839D02628DAD19F4B290028
:1048B000132218001D0007F08FF9FEF7A1FB5CE042
:1048C000712800D177E0722800D180E0602800D103
:1048D0008BE0DC28C5D1022A00D875E07378BFB21E
:1048E0006370B378A370032A05D0033A390092B2FB
:1048F000F01CFEF789FC10223900E01CFEF74AFD8F
:10490000C51C002807DA60705CE00C222000884992
:1049100006F052FF0C25280005B0F0BD013A854D88
:104920000C2A13D8002A0AD02800019906F044FF67
:10493000FFF756FE0C2228007F49FEF765FC290090
:104940000C22601C06F038FF0D25E4E70C22EBE793
:10495000784D7A4B2A0043CB43C2E9E7013A734DC5
:104960000C2A11D8002A08D00199280006F024FF4B
:104970000C2228007249FEF747FC29001322601C14
:1049800006F01AFF1425C6E70C22EDE706226D4952
:10499000601C06F011FF0625BDE712226A49601C63
:1049A00006F00AFF1325B6E708226849601C06F0E6
:1049B00003FF0925AFE77178F02905D8644B188803
:1049C00001F0B4FD0225A6E7FF236370FAE7614B0F
:1049D000012A03D072789A706270F3E79B78F4E74B
:1049E0002000FFF7E3FA050095E7013A594B5A4DCD
:1049F000072A10D8002A10D00121280059700199E7
:104A000006F0DAFE01F058F829000722601C06F0D3
:104A1000D3FE08257FE70722EEE700225A70F3E76E
:104A2000042A04D94D4D2F6006F0FEFDA860FFF763
:104A300097FD0422039003A9601C06F0BDFE052526
:104A400069E7474D062A15D906222800019906F084
:104A5000DBFE00280ED006220199280006F0ACFEED
:104A6000062240492800FEF7CFFB0123394A9178FE
:104A70000B43937029000622601C06F09DFE07255B
:104A800049E7012AA0D07078FFF772FE9AE7012863
:104A900000D0E6E6931E344F132B04D87378002B16
:104AA00009D100F015F9314B39001D78601C6A1EE0
:104AB00006F082FE2FE7551E2A000199380006F005
:104AC0007BFE2B49AAB23800FEF79EFB00F038F9B6
:104AD000E9E7DA281DD1042A00D875E7082A15D994
:104AE000B37972791B021343F27912041A43337AB1
:104AF0001B0613433B603B680522310020000393F3
:104B000006F05AFE0422601D03A950E7FE236370DD
:104B1000F1E7DE2800D057E7511E012A01D1002518
:104B2000F9E6019800F0AEFFF9E7C046A061FF1F6B
:104B30006CBD0011D461FF1FFC0C000060BD0011B2
:104B4000F50C0000AC61FF1F8C61FF1F3043FF1F9D
:104B5000F041FF1FD061FF1F8D42FF1FE061FF1F6B
:104B60006509FF1FADAC0000D163FF1FCF63FF1FBE
:104B7000AEDE000070477047020010B5094B0A32E4
:104B8000094C92B2DA815A8298811882207802F018
:104B900033FB0422054B012120781A7006F064FFD4
:104BA00010BDC046BA42FF1F1A64FF1F1964FF1FE1
:104BB000013870B5042809D806F0EEFF030928086B
:104BC0001200234B0221187806F04EFF70BD204BD7
:104BD0000821187806F040FE00221E4B1A72F5E7F5
:104BE000802200241B4B1A4D52001A8108211A689A
:104BF0002878DC7206F088FF2100287806F064FD32
:104C0000012000F05FFE00F057FFDFE7104B0821A6
:104C1000187806F021FE1048FFF766F80F4B104A8F
:104C20009B79002093800F4A13808022094B520009
:104C3000D8721A8100F046FE00F03EFF0A4B9B78C6
:104C4000002BC3D0094A136006F056FDBEE7C046EC
:104C5000F061FF1FC461FF1FF941FF1FD461FF1FF7
:104C6000BC43FF1FEA41FF1FD061FF1F34F000402B
:104C700010B501290BD1012809D1054B1B78002B58
:104C800005D02622034B04485A72FFF775FF10BD6A
:104C9000F263FF1FC461FF1FC40900000300F0B5E9
:104CA0000A4D8E18B14202D152008018F0BD0C7826
:104CB0002F6824093C5D0F271C700C7801313C40A3
:104CC0002F683C5D5C700233ECE7C046E441FF1F97
:104CD0000D22124B10B51A700C23114C1149237080
:104CE000093A033B1048637006F066FD2D2301224C
:104CF0000E490F48A371FFF7D1FF01220D49FFF7BD
:104D0000CDFF01220C49FFF7C9FF030000200B492A
:104D100002001870FEF778FA10BDC046EE63FF1F60
:104D2000CF63FF1F13BD0011D163FF1F6709FF1F72
:104D3000D663FF1F6609FF1F6509FF1FAEDE000077
:104D400070B5124C142220001149FEF723FB431EBC
:104D5000104D132B17D8AB78002B14D0431C2B709D
:104D600009236B7000230019037028782900013093
:104D7000C0B206F049FC297822000139C9B20020EE
:104D800005F0D6FD70BDFFF7A3FFEEE7D163FF1F6F
:104D9000AEDE0000CF63FF1F10B5114B1A781870FC
:104DA000002A0ED000280BD10E4B1A78062A07D8FD
:104DB0005423D340DB0703D50B4B187802F01CFAC1
:104DC00010BD0028FCD0074B1B78012B02D0033B01
:104DD000022BF5D8044B0121187806F045FEEFE7C9
:104DE000F263FF1F1964FF1F1A64FF1F70B54A4E5C
:104DF0004A4A4B493070012005F026FC00F0D8FEED
:104E0000FEF7FEF806F008FD032246494648FFF784
:104E100045FF2D24030004221C7044490130FFF794
:104E20003DFF30230470424D424C437083702E3B53
:104E3000062220004049EB87FEF7ACFA062813D083
:104E4000200006F0F9FB022809D00321200006F01B
:104E5000ABFC8D23E3706E3B237119336371062223
:104E600020003549FEF7D0F9344B1B68FC335C64F5
:104E7000FFF766FF0020FFF78FFF314C314A012119
:104E8000314B1278207802F079F9304A304B1278A1
:104E90000021207802F072F901222E4B1A702E4B5D
:104EA000DB78552B31D12D4B3B325A722C4B2D4A8E
:104EB000AB81EA812B826A822021307806F084FE61
:104EC0000120404205F080FD0120404205F01CFE1B
:104ED000FFF71CF9FEF7D0FE00F0B2FC01204042C3
:104EE000FEF7A6FF012006F0D7FCF02001F002FB40
:104EF0000121307806F0B8FD307802F0D9FA1A486E
:104F000006F09AFEFEF774FD70BD6422174B5B79C4
:104F100053431A000A32CBE7F061FF1F754B0011B3
:104F2000714C00113043FF1F8C61FF1FAC61FF1FEC
:104F3000BA42FF1F6509FF1FADAC00004464FF1FAC
:104F40001A64FF1F1842FF1FF941FF1FEE63FF1F86
:104F5000CF63FF1FC063FF1FD061FF1FC461FF1F2E
:104F6000C4090000CE090000F261FF1FD461FF1FD9
:104F7000F8B50A0020230D001A40194263D05E4B99
:104F80001B78002B5CD0FFF7EBFA5C4B5C4C5D4E62
:104F900099686268737A8A1ADB039A4202D3616065
:104FA000FEF726FD327A217A531EDBB2994205D1F3
:104FB000FFF744F9002000F0B3FD15E09142F9D36A
:104FC00000272772FFF764F9A37ABB4202D0A772C9
:104FD000FEF794FD012000F0A3FD4B4F3800FEF7D3
:104FE00083FE390006F0B0FB637A002B25D0013B2D
:104FF000DBB26372002B20D1444BDB78552B01D1FF
:1050000006F07AFBE37A002B12D00023A27AE37237
:105010009A4202D0A372FEF771FD3D4A3A4F1388BF
:10502000380001331380FEF75FFE390006F08CFB79
:10503000642370795843FFF79FFD237A013323726D
:1050400020206840F8BD0BB2002B0ADA314B1878EB
:1050500006F0D2FB002801D006F00EFB80200002F3
:10506000EFE70224214206D0254B01201A72FFF7F8
:1050700093FE2000E5E70B071ED5FFF771FA1F4BE3
:105080001F49204C98684A68637A821ADB039A4267
:1050900002D34860FEF7ACFCFFF7FAF8FFF7CEF852
:1050A000012000F03DFD00F0E5FB2368DB0701D5A2
:1050B000FEF7B6FF0820C4E7CB0609D5FEF71EFDB4
:1050C0000D4B1B78002B01D1FEF7EAFD1020B8E74D
:1050D0000124214207D0104800F06CF806F0ACFC27
:1050E00000F006FDC5E70424080020402142A9D0B5
:1050F000FEF7BAFEBDE7C046F263FF1FE061FF1F87
:10510000C461FF1FD461FF1FF941FF1FD061FF1F62
:10511000B861FF1FF061FF1FDC41FF1FF0B51B4BA3
:105120001B4F1B883A8804001A4E1B4D85B09A42CB
:105130000DD832889A420AD3184B1A882B889A4283
:1051400005D1174A174B12881B889A421BD005209D
:1051500001F026FA3B8802AA13803388019053801D
:105160002B88114D93800F4B02A91B88D3800F4BC6
:105170002A78188802F042FF0D4B08212878019AFE
:105180001C7006F0C1FA05B0F0BDC046BE63FF1F3B
:10519000EE41FF1FEC41FF1FEA41FF1FBC63FF1FF1
:1051A000BA63FF1FE841FF1F1A64FF1FF041FF1F92
:1051B000B863FF1F13B50C4B1C78002C11D10028CD
:1051C00001D00A4B18600A4A0A4B11780A4A107833
:1051D0000A4A01920A4A0092002205F0A1FA200030
:1051E00016BD1124FBE7C0461964FF1FB463FF1FFF
:1051F0001864FF1F0864FF1F1A64FF1FF463FF1F7A
:10520000F863FF1F10B5064B12201B78052B06D143
:10521000044B13221988044B187801F09DFB10BD34
:105220001964FF1FF041FF1F1A64FF1F10B500240F
:105230000122114B52421870104B1C70104B1A80F7
:1052400002F036F904220F4B21001A700E480C327E
:1052500006F0BAFB102221000C4806F0B5FB07222D
:105260000B4B1C600B4B1C700B4B1C700B4B1A70C8
:105270000B4B1C7010BDC0461A64FF1F1964FF1F42
:10528000F041FF1F1864FF1F0864FF1FF863FF1F32
:10529000F463FF1FCE63FF1FCD63FF1FF241FF1FAB
:1052A000CC63FF1FF8B5174C0600257806A8142418
:1052B0000078052D23D1B41F134FA5B21824BD4289
:1052C0001DD88D1FADB2BD4219D8FA256D00AA4276
:1052D00015D21D000D4F0A3DADB2BD420FD80C4C8A
:1052E00026800C4C21800C4900240A800B4A138034
:1052F000FFF714FF0A4B0421187806F0ADFA2000DE
:10530000F8BDC0461964FF1F790C0000750C000041
:10531000EE41FF1FEC41FF1FEA41FF1FE841FF1F65
:105320001A64FF1FF0B50BB20D0089B0002B00DB33
:1053300070E1A44E307806F05FFA041E50D0037876
:10534000A22B00D122E1D02B1AD0912B45D143784A
:105350000E2B42D19C4B82889A423ED19B4A836855
:105360001278052A39D1032018567F2835D0984B5A
:105370001B68002B31D05B68002B2ED098472CE0A7
:105380008078072829D806F007FC0428183F3F74C6
:10539000A8D86378002B0CD101218C4B19708D4B50
:1053A0001A78002A5BD08C4B307801F0E7FE002899
:1053B00055D00722854B1A7051E061780029F8D149
:1053C000E378002B11D0854A854B1278307801F0B4
:1053D000D5FE60706378002BEBD1200006F04CF90D
:1053E00080200002684009B0F0BD784B1B78022B8A
:1053F000F3D00121307806F0CFF90028EAD101215D
:10540000307806F031FBE5E76378002BD1D16F4FA0
:10541000032807D13B78052B02D101333B701EE0F6
:105420000223FBE76F4B1A886F4B0293002A0BD0C5
:105430001B78002B03D00121307806F065F93B780A
:10544000062B04D1013BE9E7029B1A70F7E7042B16
:1054500041D10121029B3078197006F005FB5C4BAD
:105460001B68002BB9D01B68002BB6D0574A1078A8
:1054700084E76378554F002B27D10622211D5B4816
:1054800006F09AF962895A4B5A491A80A2895A4BF6
:105490001A80E3890B800521397058490A80584ADF
:1054A0001380228A574B1A80574B1B78012B09D146
:1054B0001F2001F075F8FA2292004243042130784F
:1054C00006F022F90022484B75E7312B00D070E737
:1054D0000022454B1A700323A0E70622002143480F
:1054E00006F072FA0023454A04211380444A3078BA
:1054F0001380444A138006F0AFF90821307806F093
:10550000ABF9A379083B5A425341304A0333137035
:10551000304B1B78002B06D0334B30781A78002A9A
:1055200006D001F069FE0122314B52421A8096E703
:105530000121197006F098FAF5E70821307806F095
:105540008BF96378002B00D047E72C4B2D4F02934B
:10555000E388029A04211380294B3078039323892E
:10556000039A138063893B8006F016F9002800D067
:1055700033E7264B1B68002B00D12EE703990298D6
:105580003A88098800881B68984726E74379132BD7
:1055900000D022E70389012B0AD11D4B1B78022B77
:1055A00006D10821307806F057F9FFF72BFE14E7F3
:1055B000052000F0F5FF08210200307806F0A4F87D
:1055C0000BE7C0461A64FF1F051400001964FF1F93
:1055D000B463FF1F1842FF1FF941FF1FEE63FF1F57
:1055E000CF63FF1FF063FF1FF263FF1FC163FF1F45
:1055F000F041FF1FC863FF1FCA63FF1FBE63FF1F89
:10560000BC63FF1FBA63FF1FC063FF1FB063FF1FB0
:10561000B863FF1F8020C001014200D0E2E6CB0743
:1056200031D5324B1B78002B1DD0314E05AC337871
:10563000052B1AD1023B23702E4B21001B782372BD
:105640002D4B1B7863722D4B187801F03BFD002821
:1056500009D007202A4B30701B68002B03D01B6831
:10566000002B00D098470120BCE60E20254B0622D7
:105670001B7825492370254B1B78637002ABC0183B
:1056800006F09AF8D8E7022308001840194209D01A
:10569000174B1B78052B03D11D4B188806F024FAF5
:1056A00002209FE60424214203D0FFF737FD2000AB
:1056B00098E6082308001840194200D193E6154BDC
:1056C0001C78012C03D0022C0DD008208AE6124B46
:1056D000124A134913481B881288098800880094CD
:1056E000FFF7E0FDF1E7FFF78DFDEEE7F263FF1F47
:1056F0001964FF1FF241FF1FCC63FF1F1A64FF1FD5
:10570000B463FF1FCE63FF1FF341FF1FCD63FF1F75
:10571000F041FF1FB863FF1FE841FF1FEA41FF1F71
:10572000EC41FF1FEE41FF1F10B502A804880B20BB
:10573000002C10D1496808784978090201430C48C7
:10574000814209D1022119800A4B59881170DB78F6
:1057500000205BB2537010BD074C0A20A142FAD161
:1057600002211980034B998811705B79F0E7C046DC
:105770006E2A0000B861FF1F6F2A0000F7B5150000
:1057800008AA16884A680F4F1478527812022243EA
:105790000A24BA4214D10122DBB2019200962A00F7
:1057A00005F0C4FE041E0BD1074B1B68002B07D06D
:1057B00068782A78000210434242504101309847ED
:1057C0002000FEBD022900002C64FF1F30B501251A
:1057D00003790400BFB02B4225D01449408805F05E
:1057E00011FA28420CD0124B01A95B8D00220B80CC
:1057F00002234B800F4B5B888B80608802F0F4FAA9
:105800000D49608805F0FEF9C0070CD50B4B01A9C6
:105810001B8800220B8002234B80064B9B888B80C9
:10582000608802F0E1FA3FB030BDC0462464FF1F3B
:105830001C42FF1FB861FF1F1C64FF1F7642FF1F41
:1058400010B5074C0749200005F092F920000649E1
:1058500005F08EF90721054A054805F04BF910BD02
:10586000FFFF00002464FF1F1C64FF1F8CBD00119C
:105870001C42FF1F10B5024803F038F910BDC046A6
:10588000CD5700110221430888400B400A310840DF
:1058900003430E20024AD17881430B43D3707047F3
:1058A0008D42FF1F064A1379410705D580210B431E
:1058B00080011371907170477F210B40F8E7C0465B
:1058C0008D42FF1F054A5378002803D080210B43E7
:1058D000537070477F210B40FAE7C0468D42FF1F8F
:1058E0000F21114BDA780A40DA70502810D90131B3
:1058F0000A43DA702022D9780A43DA704022D97834
:105900000A43DA708022D97852420A43DA7005E0FD
:105910003C28EFD82828F1D81428F3D80122D978C8
:105920000A43DA707047C0468D42FF1FF8B57F23E7
:10593000324D04006E789E43314B984205DD76234C
:105940002B70363B33436B70F8BD2E4B984203DA15
:1059500058232B701433F5E783B21A0000215F320D
:10596000294892B2294F297082422DD9A9708C42C0
:1059700003DA5B421CB220232B70053420B20A21CB
:1059800005F0F2FF04B2FA239B009C4233DB802334
:105990002A785B4213432B706421200005F0E4FF5A
:1059A0000A2100B205F0E8FF09B22A787B5C1343B4
:1059B0002B700A21200005F0D7FF0A2100B205F064
:1059C000DBFF09B27B5C0AE08022AA70002CDADAE5
:1059D0005B421CB220232B705F23092CE9DC1E43A1
:1059E0000A2120006E7005F0C7FF09B2AA787B5C1F
:1059F0001343AB70A8E7632CCEDCEDE78D42FF1FAD
:105A00001B4E00001DFCFFFF2A080000B6BD001160
:105A10007F23F7B5194FCD013E7904009E433E71B7
:105A2000EDB2632806DD093B33433B7140231D4340
:105A30007D71F7BD0300093304DA582333433B710A
:105A40006C23F4E70E4B019300280BDA0423444245
:105A500024B23B710A21200005F08EFF019B09B2A0
:105A60005B5CE4E70928F5DD0A2105F07DFF019B79
:105A700000B21B5C1E433E71ECE7C0468D42FF1F27
:105A8000B6BD0011F8B50A4F05003B780E00002B9B
:105A90000CD0084C2000FEF72DFC33002A0020001B
:105AA0003978FEF71BFD2000FEF762FCF8BDC0460A
:105AB0003864FF1F9442FF1F70B50A4E0A4D07223B
:105AC0003100280005F0A0FE002809D0074C310065
:105AD0000722280005F070FE08212000FFF7D2FF02
:105AE00070BDC0468D42FF1F3164FF1F3064FF1F31
:105AF0007F207C2210B5094B59781A708143103AE7
:105B00000A435A7078220E219A70DA7858718A43C3
:105B1000DA7006221A71FFF7CFFF10BD8D42FF1F0A
:105B200010B5002832D01E4C0223E05E1D4B1B68CE
:105B30005B062CD509233221584305F015FF41306F
:105B4000FF3000B2FFF7F2FE0520FFF79BFE0422B4
:105B5000A35E154A6320934205DC323318006421AA
:105B600005F002FF00B20121FFF752FF207AFFF794
:105B7000B7FE0020FFF796FE0C4B1878053843421D
:105B80005841C0B2FFF79EFEFFF796FF10BD0A21F5
:105B9000053005F0E9FE00B2FFF7C8FE0320D4E7A8
:105BA000B861FF1FD461FF1FDD2600001964FF1FCD
:105BB00070B50024094D2800AC71FEF79BFB102343
:105BC0003E212800064AFEF789FCA04200D13E345F
:105BD000044B28001C70FEF7CBFB70BD9442FF1FE6
:105BE000A6BD00113864FF1F0200F0B501270A4866
:105BF0000A4E51188B1A002B00DCF0BD08241578D2
:105C00004308684038404000805B013C58406D08C4
:105C1000002CF5D10132EDE7FFFF0000C6BD0011F9
:105C2000F0B500250F269D4200DBF0BD4C5D070955
:105C300044403440A400A05801357840F3E7000008
:105C4000F0B589B06A460D000B000F271100103522
:105C50001C780133260024093E401670547002322D
:105C6000AB42F5D12023024AFFF7DAFF09B0F0BDBD
:105C7000CCBD0011F0B54E780B7889B036020C001F
:105C8000170001901E43012A61D9954B9E4200D80E
:105C900077E001339E421CD1062A17D1CA788B784F
:105CA00012021A430B791B0413434A7912061A4352
:105CB0008C4B5A6100221A705A808B4A5A608B4A68
:105CC0009A608B4ADA60002009B0F0BD8822520544
:105CD000EEE7884B9E423CD182498B78002B00D066
:105CE000F6E00C2A31D10F22A3789343E278120216
:105CF00013432279120413436279120613434B6053
:105D0000E279A07912020243207A00041043627AF9
:105D100012060243CA60E27AA07A1202024376486F
:105D20004A81834208D804236E49142201980B70DB
:105D300005F042FD1420C7E71201D21889235B0544
:105D40009A42F0D801238B70BDE7022AFAD00523CE
:105D5000EAE76A4A01239642E6D1FFF753FA052F94
:105D60000CD9E378A2781B021343227912041A4358
:105D700063791B061343624A0393136005F0BCFC6E
:105D8000A1E7584D2B78002B9DD1AB78002B00D18B
:105D9000A0E02B8901339BB20093B34200D091E085
:105DA000132AD4D9CF7C8B7C3F02122120001F43C1
:105DB000FFF71AFF874200D08EE0002E3DD1E37836
:105DC000A2781B0213432279E96812041A4363790B
:105DD0001B06134303930A228B4212D1FF23A370A5
:105DE000E370237163716B89002B09D1E37B227C03
:105DF0001B0212041343A27B13431B0901336B8163
:105E000000226B89002B8ED0002A67D16868370189
:105E10003818000B6B6900030390984205D968613C
:105E200005F062FDEB780133EB7068681022A11C6D
:105E3000381805F049FD2E8145E76F89009A7B1ED1
:105E40009BB293423AD1E278A37812021A432379A3
:105E500005A81B04134362796C6812061A43EB68A9
:105E600000920392211D0C22049305F0A5FC012051
:105E7000260004A940421036FFF7E2FE013F012F41
:105E800017D1009A0B232861824200D04CE70422EC
:105E90001C49200005F018FD042203A9686805F0DC
:105EA0004BFDE968039AFF23914200D13CE7F73BA1
:105EB0003AE73100FFF7C4FE1036DFE70923B742A7
:105EC000A4D831E7009BB34200D9FCE607232BE7B7
:105ED000022329E7032327E7062325E70A2323E7ED
:105EE000FFFE00009C42FF1F00000111FFFF0000A9
:105EF0005048593601FF0000FFFF001102FF00006B
:105F000034F00040A842FF1F10B5034C0B000122E3
:105F1000210000F06BFA10BDC96000110B8870B54C
:105F200006000D000224162B11D92B00032209496B
:105F300000F05CFA041E0AD1074B2A881B88191C42
:105F4000934200D9111C300089B200F0EFFA200012
:105F500070BDC046F56000114A64FF1F10B54A7855
:105F60000400013A0B000220012A07D80A78002A0F
:105F700004D005222000024900F038FA10BDC046C6
:105F8000236100110A7810B50B0004000220002ADA
:105F900004D007222000024900F028FA10BDC046B4
:105FA000CF6100110A7810B50B0004000220002A0E
:105FB00004D009222000024900F018FA10BDC046A2
:105FC0003562001110B5034C0B000B22210000F0CC
:105FD0000DFA10BD6562001110B5034C0B000D22C7
:105FE000210000F003FA10BDD762001110B5034C78
:105FF0000B000F22210000F0F9F910BD31630011F0
:106000000A7810B50B0004000220002A04D01122E7
:106010002000024900F0EAF910BDC04641630011BA
:10602000002310B51322190000F0E0F910BD0000A4
:1060300010B5034C0B001722210000F0D7F910BD5A
:1060400093630011002310B51922190000F0CEF956
:1060500010BD000010B5034C0B001B22210000F006
:10606000C5F910BDCD630011F7B584890D00060098
:106070000121002C22D000238268D3561778002BF0
:106080001EDA0C2C1AD90C3CA4B2131940880093C8
:10609000230002F086FE431E984101307B06DB0F91
:1060A0006B703F23013C1F40A4B22870AF70AC80DE
:1060B000002C07D0B3680133AB6000210800FEBD9F
:1060C0000020EBE7AC60F8E70B7803704B88437077
:1060D0004B881B0A83700B79C3700420704704201F
:1060E000022B06D10020537811781B02009A0B4333
:1060F000138070470B8803700B881B0A43700220C3
:1061000070470420009983420AD1537810781B020B
:1061100003430B80D37890781B02034300204B800D
:106120007047F8B50D004B7801240021461C037020
:106130002B788B4201D82000F8BD6B78B01C4F1C27
:10614000012B10D1890069184B88022233704B88CB
:10615000B9001B0A7370691805F046FC0436043454
:10616000A4B2F9B2E4E7122359436B185A880431F8
:1061700032705B8810221B0A7370691805F034FCBA
:1061800012361234ECE770B5049D14001E00052B86
:1061900001D8042070BD637812781B0213432B8052
:1061A000E378A2781B02134302226B802A71211D1F
:1061B000681D063E05F018FCB2B22A81E92AE8D82B
:1061C0002800A11D0A3005F00FFC0020E2E70023A3
:1061D00010B50A789A4201D8900010BD9A008A182A
:1061E0005488013304705488DBB2240A44709488C4
:1061F00084709288120AC2700430EAE710B5110068
:10620000029C062B04D004201022142B01D010BDB8
:10621000022222714B7808781B0203432380CB783B
:1062200088781B02034363800431601D05F0DCFBAA
:106230000020ECE710B50C788B7804315C43E4B2B5
:1062400003702200013005F0CFFB601C10BD04205C
:10625000022B06D10020537811781B02009A0B43C1
:106260001380704710B50C000A88023105F0BCFBA2
:10627000208810BD70B504000D0004981100012B9A
:1062800001D8042070BD1678527812023243028081
:106290000200F13255701470E125002C00D10C354C
:1062A000023B9AB24280AA42EBD80231043005F098
:1062B0009BFB0020E6E70420009983420AD1537833
:1062C00010781B0203430B80D37890781B020343A2
:1062D00000204B80704710B50C000A88023105F091
:1062E00083FB208810BD000070B501211E00042032
:1062F000049C0E400B4218D1CB40DDB28D4214D924
:106300000A49DBB2098899420FD32300EE331D708E
:106310003300580011184978165C090231430133E3
:106320002152D9B28D42F4D8002070BDB442FF1F73
:1063300010B50C000A88023105F056FB208810BD0C
:1063400010B50C788B7804315C43E4B20370220002
:10635000013005F049FB601C10BD10B5110002981A
:10636000032B01D8042010BD14785278043B12028C
:1063700022430280CA788C781202224342809AB269
:106380008280EB2AEED80431063005F02DFB002088
:10639000E9E710B50C000B8803700B881B0A4370EB
:1063A0004B8883704B881B0AC3708A88043006317F
:1063B00005F01AFBA088043080B210BD0420012B28
:1063C00003D100201378009A1370704710B50C00A9
:1063D0000B8803700B881B0A43704A880230043113
:1063E00005F002FB6088023080B210BDF0B589B0C4
:1063F00003931E4B029242000700D05A019102F013
:1064000020F81325061E2DD0029B01240370019B4A
:10641000002B04D0001903999847001984B26B46E9
:106420001B7A5BB2002B0FDA1021380002F01CFB44
:106430001925002813D130003219E1B202F066FCB0
:10644000051E0CD10C34A4B2042304AA380005A9FB
:1064500093800696948101F0AFFD051E02D03000B6
:1064600005F062F9280009B0F0BDC0464864FF1F7E
:1064700070B505000C0000280CD00020814209D026
:1064800010222000044905F0AFFA01202B78237375
:106490006B78637370BDC0460CBE0011F0B506008A
:1064A0000D0017001C0085B002291BD00020102908
:1064B00007D1022B07D0102B03D115E00020102CA0
:1064C00008D005B0F0BD69463800FFF7D1FF2A00BB
:1064D00069460BE069463000FFF7CAFF22006946B3
:1064E000380004E0022BE9D12A003900300005F021
:1064F0001BFBE6E7031CF02800D9F0230320084922
:106500009AB2013A0B80D317034006499B189B109F
:106510000B80D30F04499B185B100B807047C0465B
:10652000B842FF1FB642FF1FB442FF1F034B1B8838
:106530008B4202D3024B4000C1527047B842FF1F4A
:106540004864FF1F014B4000185A70474864FF1F02
:106550001722014B1A8070474864FF1F70B5050071
:106560000E2005F001F9041E13D0D0230370002380
:106570000622837007494570033005F035FA064B53
:106580002100DA8A62811B7E2373044B187805F0A0
:1065900003FA70BD6464FF1F5464FF1F0843FF1FAC
:1065A000262803D8024B4000C05A70470148FCE738
:1065B000BA42FF1FFFFF000070B506000C00094D36
:1065C0001C220021280005F0FFF9074B1E70074B25
:1065D0001C7005F009F90123002801D000231220C6
:1065E0002B7070BD5464FF1F0843FF1F7564FF1FAD
:1065F00070B505000D4C0800E260A160102200217A
:10660000656005F021FB012803D11021A06802F08C
:1066100058FD10220021280005F016FB012803D1A7
:106620001021606802F04DFD70BDC0465464FF1F2C
:1066300070B5041E05D1002903D006220D4805F0CF
:10664000D3F90D4B1D78012D11D1002C05D102225B
:106650001A7005F0E9F8280070BD00221A70074B87
:106660001B78FF2BF7D02000FFF778FFF3E700251A
:10667000F1E7C0466464FF1F5464FF1F0843FF1F17
:10668000030010B5002801D1002010BD00780B4A8E
:10669000002803D15988D1821B7913761378022BF5
:1066A000F2D10023984200D103331370044B1B78BE
:1066B000FF2B01D0FFF752FF0120E6E75464FF1FD4
:1066C0000843FF1F002911D000280CD04B79012866
:1066D00003D140225242134303E03F2213400328D8
:1066E00002D001204B7170474022F4E70800FAE71E
:1066F00070B5094D0100287800280BD0074C062200
:10670000200005F071F921002878FFF7DBFF200059
:1067100005F052FA70BDC0467464FF1F4E64FF1F3F
:1067200000290AD0012808D13F224B799343C02B7E
:1067300003D0403B5A425341981C704770B5174DE7
:1067400006002B78FF2B15D00A2005F00DF8041E4B
:1067500010D0D0230370C83B8370114B11491B78B4
:106760004670C3700622043005F03EF921002878F7
:1067700005F012F90C4B1B78012B0DD10B4B1B684C
:10678000002B03D09B68002B00D09847084B0421B6
:106790001878084A05F0B8F970BDC0460843FF1FD5
:1067A0007464FF1F4E64FF1F7064FF1F9C64FF1F13
:1067B000A064FF1F60EA0000014B98687047C04664
:1067C0005464FF1F014BDB68186870475464FF1F57
:1067D000074B10B5DA68136801331360054B18785E
:1067E000FF2803D08021C90105F03EF910BDC04645
:1067F0005464FF1F0843FF1FF7B50E0002F0C8F8EE
:10680000051E1CD00E4B06621F78002F00D10778A2
:10681000AB791020019304F0A7FF041E0FD0D02302
:106820000380C73B8370019BE91DC37006220430BF
:1068300005F0DAF821003800E66005F0ADF8F7BDA4
:106840000643FF1F014B18787047C0467464FF1F52
:10685000054B002805D1054B1A78054B002A00D1BD
:10686000014B18007047C0466464FF1F7464FF1F2B
:106870004E64FF1F014B58687047C0465464FF1FA9
:10688000024B1868431E9841C0B270477864FF1FDE
:10689000421E03000120152A03D9FF3B5A425341EF
:1068A000D8B27047F0B51C0000230E0085B00390ED
:1068B00002920B70029A934201D3002019E0E55C2A
:1068C0005A1CD2B2002DF8D0029851198142F4DC42
:1068D0000233DFB2A35C18000193FFF7D9FF002851
:1068E00007D0013D019A0399EBB233708A4202D17D
:1068F000E01905B0F0BDDB19DBB2DBE710B50C0029
:1069000002F09EF803001220002B03D021005888CB
:1069100004F0A2FE10BD000070B50E4D8400635956
:10692000002B15D0186A002801D004F0BDFE2B59A9
:10693000586A002801D004F0B7FE2B59986A002845
:1069400001D004F0B1FE285904F0AEFE00232B5113
:1069500070BDC0468464FF1F1C4B70B504000E0060
:10696000150099420AD11A4B1B68002B01D1122045
:1069700070BD1B68002BFAD09847F9E7154B994278
:1069800015D1134B1B68002B0AD01B68002B07D0B6
:106990009847002804D1104B1C70104B1D70E7E77E
:1069A00029002000FFF7AAFF0028E1D1F3E7080043
:1069B00001F0EEFF0028DAD003780320A342D7D1FC
:1069C0002900300004F048FED2E7C046FEFF000078
:1069D0008064FF1FFFFF00007D64FF1F7C64FF1FBA
:1069E000F7B50400808801F0D3FF0025A84203D04A
:1069F0000578A08802F008F81C4E3378002B1FD0D1
:106A0000AB421DD11A4B28001978FFF777FF0028F9
:106A100018D000233370A3790820A778A6880193A3
:106A200004F0A2FE011E0DD0D0230370CA3B837078
:106A3000019B477086808371280004F0ADFF01E060
:106A4000002DE8D1A0880B4B8200D358002B01D039
:106A5000FFF762FF1721A088FFF768FDA08801F00B
:106A600027FDA08801F0FEFDF7BDC0467D64FF1F35
:106A70007C64FF1F8464FF1FF0B587B01D000CAB62
:106A80001B88070001930DAB1B88142002930EABEB
:106A90001B88160003930FAB1B880091049310AB67
:106AA0001B88059304F060FE041E1AD0D0230370E7
:106AB000CB3B47708370C670062229000430002D3E
:106AC00011D004F091FF019B21006381029B00988B
:106AD000A381039BE381049B2382059BA37404F0A1
:106AE0005BFF07B0F0BD04F06FFFECE7F7B5009374
:106AF00008AB1B8807000C200D001600019304F062
:106B000033FE041E13D0280001F042FF00280FD0EE
:106B10000078D0232370C93BA370009B2100238100
:106B2000019B6770A580E680638104F035FFF7BDA7
:106B3000014B1878EDE7C0460843FF1F13B504006A
:106B400064890389C2888188C0780094FFF7CEFFEA
:106B500013BD000010B5044C2068002803D004F0D9
:106B6000A3FD0023236010BD8864FF1FA122F0B5A0
:106B7000818892004A43384B384F1B6804009B18A9
:106B80009D2292009B18827989B01A603B68002B85
:106B90005FD01D78324B1B68002B04D05B68002B44
:106BA00001D000209847260008363100E079FFF731
:106BB000B7FD237DE0710200E0780493638A290029
:106BC0000393238A0293E3890193A38800933300FC
:106BD000FFF752FFE378002B0BD1E289A379A1885C
:106BE00002920196E27928000092012201F0DAFE79
:106BF000E0703B68002B20D0FFF7ACFF194D2878E0
:106C000000281AD0184B1978FFF778FE002814D006
:106C10002B78E67808200793A78804F0A5FD011ECD
:106C200009D0D0230370CA3B467083708780867179
:106C3000079804F0B1FE00232B701721A088FFF7FE
:106C400075FCA08801F034FCA08801F00BFD09B0B0
:106C5000F0BD064B9DE7C0463409FF1F8864FF1F47
:106C60009C64FF1F7D64FF1F7C64FF1F0843FF1FA0
:106C7000F8B5070008000E0001F08AFE041E18D0C7
:106C80002620FFF78DFC051E00D12578062004F094
:106C90006BFD041E0DD00021062204F095FED023CA
:106CA0002370C23B21006770A370A680E8B204F095
:106CB00073FEF8BDF0B585B001930AAB1B780700F1
:106CC00002930BAB1B7808000D000092039301F0B8
:106CD0005FFE061E22D0102004F046FD041E1DD0CB
:106CE0001022002104F070FE2620FFF759FC002836
:106CF00000D13078D0232370C13BA370009B2100CA
:106D00002372019B67706372029BA580A372039B31
:106D1000C0B2E3720C9BE36004F03EFE05B0F0BD30
:106D2000F7B50D00019001F033FE071E20D00E20B4
:106D300004F01AFD041E1BD02620FFF731FC061EAE
:106D400000D13E78D0232380C53B0622A370F91DD5
:106D5000E01C04F049FE019B2A0063810123DD4011
:106D60001A401D40210022736573F0B204F014FE36
:106D7000F7BD0000F0B585B0029010000D001700BF
:106D80000A9E039301F004FE041E31D0029B002BE7
:106D90002ED1039B02795B0724D5122313430422CF
:106DA000002E08D10B99002905D10C99002902D198
:106DB0000D9900291AD01A430D9B2271002B00D087
:106DC000C9E0002E00D1CFE0002D00D0CCE0606AF9
:106DD000002801D004F068FC1C21300004F054FDB0
:106DE000606205E002239A430E33D7E79343237191
:106DF000654BBA00D458002C00D1AAE0002E10D068
:106E0000236A002B03D11C2004F056FC20625E4B49
:106E1000BA00D358186A002803D01C22310004F0AD
:106E2000E3FD0C9B002B12D0574CBB001D596B6A25
:106E3000002B03D1162004F03FFC6862BB00E3582E
:106E4000586A002803D016220C9904F0CDFD0D9B42
:106E5000002B11D04C4DBC006659B36A002B03D1F6
:106E6000142004F029FCB0622B59986A002803D042
:106E700014220D9904F0B8FD380001F089FD051EBB
:106E800067D0414BBA00D358002B62D01A6A342025
:106E9000002A00D11C389A6A002A01D0143080B22E
:106EA0000B9A002A01D01C3080B25B6A002B01D003
:106EB000163080B204F058FC041E4AD0182200217B
:106EC00004F082FD2620FFF76BFB0190002801D122
:106ED0002B780193D0232370029B200063700A2338
:106EE000294EA370039BBD00A371AB59A780196AFB
:106EF0001830002905D01C22A06004F075FD200088
:106F000034307359996A002907D0030014221433CE
:106F1000E060029304F068FD02980B9B002B08D000
:106F200003001C221C330B992061029304F05CFDCA
:106F300002987359596A002903D01622606104F03F
:106F400053FD6B462100187904F026FD3800FFF749
:106F5000E3FC05B0F0BD10220D9B0D991B69A01834
:106F6000236204F041FD2CE70B9B002B00D13FE78F
:106F7000012D00D03CE7606A002801D004F094FBAA
:106F80001C210B982AE7C0468464FF1F10B5044CEF
:106F90002068002803D004F087FB0023236010BD85
:106FA0007864FF1F0B4B07B51A68002A01D1002037
:106FB0000EBD6946531C012012780731FFF772FCA1
:106FC0000028F4D002780123100018401A42EED0B5
:106FD000EEE7C0469464FF1FF0B51F4F01203B68E9
:106FE00087B0002B25D09B78059300F0B3FB0028D9
:106FF00021D00A20FFF7D4FA04000B20FFF7D0FAC3
:10700000164B05001E78731E9E413B68F6B2191D93
:10701000D878FFF757FB3B682900DA7A04330392EC
:107020009A7901930292009033002000059A04F0AF
:10703000BBFD07B0F0BDFFF7B5FF002805D0062067
:10704000FFF7AEFA04000720D8E70820FFF7A8FAF8
:1070500004000920D2E7C0467864FF1F7464FF1F54
:1070600070B50A4E040033780D00FF2B0DD00420BC
:1070700004F07AFB011E08D0D0230370CE3B45708C
:107080008370C470307804F087FC70BD1843FF1F14
:1070900070B5040006200D0004F066FB011E0AD046
:1070A000D0230370CD3B8370054B44701B688580F3
:1070B000187804F071FC002C01D0FFF767FF70BD59
:1070C0007864FF1FF8B5264F06003B680D001124B9
:1070D000002B05D10522234B1B78134202D1122429
:1070E0002000F8BD204A10241268002AF8D0127837
:1070F000002AF5D0DB0719D52B789A1E012A1AD859
:107100000C2004F0D9FA132438600028E8D00023BA
:107110000A22437029000670023004F065FCFFF774
:107120005BFF041E0AD0FFF731FFD9E700F012FB26
:107130000028E1D1E4E7002BE2D0D0E70B4B1B782D
:10714000032BCDD11D20FFF72BFA094B1880002807
:10715000C6D0084B04211878074A04F0D5FCBFE7D5
:107160007864FF1F7564FF1F9464FF1F7464FF1F22
:107170007264FF1FA064FF1F60EA0000F7B501936F
:10718000194B14001A78052306000F0012201A422A
:1071900021D0012920D1154B1D68002D1BD00220C4
:1071A0001F2C18D8002C02D0019B002B13D0104BA1
:1071B0001F221E706E1C0021300004F005FC019996
:1071C0002200300004F010FC310020002C70002F51
:1071D00006D004F099FBFEBD064B12201D68DCE7CB
:1071E00004F012FAF7E7C0467564FF1F9464FF1FAE
:1071F0001843FF1F9064FF1FF8B50F4E1224336829
:10720000002B17D01B780F3C834213D100250B4F66
:107210000221387804F020FB094B042138781D80C6
:1072200004F01AFB074B28001D8033685C7004F0E3
:10723000EBFB04002000F8BD7864FF1FA064FF1F73
:107240008C64FF1F7264FF1F70B5012823D11B4C93
:107250002388002B03D01A4A1578002D07D0194B2C
:107260001B68002B02D01878FFF7C6FF70BD3B2BC0
:1072700002D93C3B2380F9E7134E0221307804F019
:10728000EBFAFA222388920002215A43307804F064
:107290003BFA2580EAE70B4B1B68002BE6D00B4B33
:1072A0001B785B07E2D5084B0221187804F0D4FA6A
:1072B0000022024B1A80FFF769FED7E78C64FF1F9C
:1072C0007064FF1F7864FF1FA064FF1F7564FF1FB9
:1072D000F8B51E4D2868002803D004F0E5F9002316
:1072E0002B601B4E3068002803D004F0DDF900232A
:1072F0003360184F05243B7818002040234221D0EA
:10730000154800F02BFA3B78234213D0202004F0DC
:10731000D3F92860002813D02022002104F054FB68
:10732000202004F0C9F9041E306005D0202200217D
:1073300004F04AFB002004E0286804F0B5F92C6052
:107340001320F8BD00F00AFAF4E7C0469464FF1F6A
:107350009064FF1F7564FF1F0C43FF1F10B50A4C9C
:1073600023681A1E0ED0002808D10130587004F08E
:107370004BFB002805D02368002B02D00021FFF72B
:1073800087FE0122100010BD7864FF1FF7B5274E5D
:10739000050033680191181E21D05C78244F012C20
:1073A00030D1FFF7FFFD002825D02000FFF7F8F8C7
:1073B0000400412814D91F4B022118781E4A04F0FA
:1073C000A3FB1E4B3C3C1C80022233685A703B7866
:1073D000002B14D128000199FFF75AFE0120FEBDB1
:1073E000FA2292004243002AEED0124B0221187872
:1073F00004F08AF9E8E7FFF7D3F80200F3E7002387
:107400003B70EBE73B78002BE8D1032004F0ACF9AC
:10741000011E08D0D0230370CC3B457083703368C5
:10742000187804F0B9FAFFF7B1FDD7E77864FF1FC9
:107430007064FF1FA064FF1F60EA00008C64FF1FE0
:1074400010B51749838802008B4220D011D8154906
:107450008B4217D0144900205B1899B2012907D834
:10746000926811785A425341D8B2FFF7F9FD0120D2
:1074700010BD0E4A00209B1807229BB29A42404141
:10748000C0B2F5E783681878FFF768FFF0E7836814
:1074900099785A78090218781143FFF777FFE7E7E0
:1074A0000A20000006200000F8DFFFFFAFDFFFFF2B
:1074B000014B18707047C0461943FF1F10B5064CAA
:1074C000207001F041FA207804F06EFA052120784E
:1074D00000F062FD10BDC046A064FF1F0BB273B583
:1074E0000D00002B00DBC4E0884B187804F084F911
:1074F000041E0ED00378912B0FD0A22B00D1A1E057
:10750000834B1878FF2852D0210004F045FA002858
:107510004DD180200002684076BD43780F2B76D095
:1075200013D8052B70D00E2BEAD18088794B984266
:107530002BD8794B98421BD8784B9842E0D1A3685E
:107540001878591CFFF774F838E03E2BD8D18378AF
:10755000032B74D06CD8012B6ED0022BD0D1704B82
:107560001B68002B23D05B68002B20D098471EE0BF
:107570006C4BC0180C28C3D804F0A6FA1DC2C21563
:107580000BC20B0B0B3223C23C00674BC018072801
:10759000B6D8664B1B68002B09D01B68002B06D0A1
:1075A000200098470AE0A3681878FFF7C7F8200082
:1075B00004F062F8ADE7A068FFF762F800289FD0FA
:1075C000F5E7A3681B78002BF1D0554B1B68002B07
:1075D000EDD01B68002BEAD0210055489847EDE715
:1075E0004F4B1B68002BE2D01B68002BDFD0210023
:1075F0005048F3E7504B1B68002BD8D05B68002B3A
:10760000D5D021004348E9E7FFF7EAF9CFE78088C2
:107610004A4B984203D04A4B984200D070E7464B01
:107620001B68002BC3D05B68002BC0D02100D5E7BE
:10763000153B012BBBD963E7FFF798FAB7E7FFF7D4
:107640007DFAB4E73F4B1B78042B07D100236A4631
:1076500013800179408800F0C5FCA8E7364B1B6811
:10766000002BA4D05B68002BA1D0010036489847BE
:107670009DE7012421420AD0294B1B68002B04D02E
:107680005B68002B01D000209847012043E78B075F
:107690000AD5264B1B68002B04D05B68002B01D059
:1076A00020009847022036E70421280008400D42B8
:1076B00000D131E7254E3388002B21D0013B9BB20E
:1076C0003380002B1AD1FFF7DBF800280AD0204BBB
:1076D0001C70164B1B68002B04D05B68002B01D07C
:1076E00020009847FFF7C6F8694601F001FD68469B
:1076F000FEF7FEFF1D20FEF753FF308004200AE74F
:10770000024B187804F0A8F8F8E7C046A064FF1F01
:107710001943FF1F0E200000012000000910000087
:107720009864FF1FFEDFFFFFAFDFFFFF9C64FF1FBA
:107730000C2000000B2000008064FF1F0D200000C3
:10774000132000007564FF1FFFFF00007264FF1F1D
:107750007064FF1F10B501F09BF910BD014B18605C
:107760007047C0469C64FF1F0B880020162B01D871
:1077700017230420014A13807047C0464A64FF1F44
:1077800000207047074A03001188814207D0918882
:107790000020994202D1013080001018704700206B
:1077A000FAE7C046A864FF1FF0B58F7806000D0009
:1077B000C5B01E2F15D1FFF7E5FF051E03D100242C
:1077C000200045B0F0BD00223B003100C07800929F
:1077D00000F0B2FB0400A81C00F0D2FBFF23EB700A
:1077E000EEE7264B062403931B78FF2BE8D0182FD7
:1077F000E6D87B08224A013BDB0002929A58944665
:10780000002ADDD0029AD3185B68002BD8D0087804
:10781000002802D14B78012B02D10624122FCFD1A0
:1078200007AFAB88697800976446AA68A047041E32
:10783000C6D1AB78029A5B08013BDB00D318390054
:1078400030005B689847041E0BD1AB78042BB6D090
:10785000039A310010782200009700F06DFB0400BD
:10786000AEE76A78002AABD1AA7805A93B880871EF
:1078700030000A704B80FEF747FBA0E71C43FF1F58
:107880001CBE00111D4B37B5050098420BD00029D6
:107890000AD1FFF777FF002805D11948FFF772FFDB
:1078A000002800D0058037BD01291AD1FFF76AFFF3
:1078B000041EF8D001235B420380A378FF2BF2D093
:1078C000FE2B07D00023E0781422009329001E33FA
:1078D00000F032FBA01C00F053FB01235B426380ED
:1078E000E1E70229DFD1013901F0BEF80028DAD141
:1078F0002800FFF747FF041EDFD1D4E7FEFF00009A
:10790000FFFF0000022210B5074B52421A800748C1
:1079100001325A809A80DA8000F07EFA044801F041
:1079200025F8002010BDC046A864FF1FA9770011EC
:10793000857800110388F7B50400002B02D10225D9
:107940002800FEBD42680221137825485268FEF7E0
:10795000A5FD00282ED0234F01253A88002AEFD01C
:10796000802321885B0201259B1A9942E8DC0C20C8
:1079700003F0A2FE061E31D03B8822889C460023DD
:107980001800019561469DB2491989B2AA421BD8D7
:10799000002801D062443A8000233000082208C049
:1079A000210004F021F8104A1368002B13D10025A0
:1079B0001660C5E76268022113780C485268FEF72A
:1079C0006DFD0028C7D1BAE760681D0140194181EB
:1079D00001330198D6E71A001B68E6E71325AFE7E5
:1079E0008ABE00111A43FF1FA464FF1F88BE001146
:1079F000014B18707047C0461C43FF1F14230A0038
:107A000010B51A40194204D00122102101F048F8A3
:107A100010BD4B06F9D4012088434000F8E710B5AB
:107A200014008B0604D50122102101F039F810BD95
:107A300008230A001A40194202D14BB2002B0FDA78
:107A4000102101F02DF8002808D02300F2331B7814
:107A5000002BECD0F1342378012BE8D10020E6E7AD
:107A600003208907FAD4E2E7F0B51F00184B85B070
:107A70001C68019002910392002C27D1200005B0D0
:107A8000F0BDA5683301ED186B89019A934211D3BB
:107A9000029A93420ED8002F04D10A9B002B10D1DA
:107AA0002C00EBE73B002978039A6868FEF7F6FCA8
:107AB0000028F2D10136B6B2A388B342E1D82468D7
:107AC000DAE7A3680A9A5B891380E9E70026F3E7FF
:107AD000A464FF1F37B50C000A884988012391422E
:107AE00017D3002A15D0651D23792A0002210A48E0
:107AF000FEF7D4FC102300280BD02379618820885E
:107B000000242A000094FFF7AFFF0A23A04200D010
:107B1000230018003EBDC0468ABE001113B50A00FE
:107B200008884988012388420BD8002809D00024FE
:107B3000137905320094FFF797FF0A23A04200D083
:107B40002300180016BD13B50A00088849880123D0
:107B500088420BD8002809D00024137905320094FC
:107B6000FFF782FF0A23A04200D02300180016BDB1
:107B7000F0B58BB003904A8808880E00012382423A
:107B800055D3002853D00023012704AC23700022D2
:107B9000718813000092FFF767FF051E3ED0207822
:107BA000002835D12B78022B18D167706A898300A1
:107BB0000130E31880005A8069680222201803F01F
:107BC00013FF23780133DBB22370042B19D93B0058
:107BD0006889013080B2002BD9D01FE00223637086
:107BE000122358436A89231804305A806968102286
:107BF000201803F0F9FE23780133DBB22370002B49
:107C0000E5D10C4A6B899B185A425341DBB2DFE73E
:107C10006378012BE4D12B78022BC7D022780A237A
:107C2000002A04D021000398FEF798F900231800D9
:107C30000BB0F0BD0100FFFF0F4BF0B5040018685A
:107C4000002816D083685D89A54207D88288AE18BF
:107C5000B44203DA12019A18934201D10068EFE7A7
:107C60001E005F891036A74204D1002900D00D8084
:107C70001800F0BD3300EFE7A464FF1F70B50500E6
:107C80000C0008880021FFF7D7FF03000120002B1C
:107C900004D022002800197AFFF7C1FE70BDF7B5A5
:107CA0000C00002501902300EE331B78AB4201D875
:107CB00000200AE06B00E65A00213000E718FFF7C9
:107CC000BBFF002802D126800130FEBD017A019859
:107CD000FFF794FE002802D03B882380F5E70135AA
:107CE000EDB2E0E710B5040008880021FFF7A4FF1B
:107CF00003000120002B03D02000197AFFF77EFE3D
:107D000010BD0000054B1B68002B01D1180004E0DA
:107D10009A6852898242F6D198887047A464FF1FFE
:107D2000F0B50E27002687B0039302ABFF183E8004
:107D300005001F4B40891400984207D02B78013072
:107D400000976A6880B2FFF78FFE060002212B7849
:107D500018486A68FEF7A2FB00280FD06C89200043
:107D6000FFF7D0FF002802D0013C0419A4B2039B06
:107D7000002B00D01C80300007B0F0BD02212B7812
:107D80000D486A68FEF78AFB0028E7D102212B78AC
:107D90000A486A68FEF782FB002807D0002EDED072
:107DA0003B88A342DBD17489013CDFE76C89DEE7C5
:107DB000FFFF00008ABE001188BE001186BE0011C0
:107DC00010B50C00FFF7DEFC03000220002B0AD0E8
:107DD000002C00D023609B781720FE2B03D00138A5
:107DE000FF2B00D1002010BD73B50D0001A90400C8
:107DF0001600FFF7E5FF172805D0002E04D1290053
:107E00002000FEF727F976BD01221021200000F0A6
:107E100047FE0028F3D0F6E7014B18607047C046D4
:107E2000B464FF1F37B56B469D1D0100040002229C
:107E3000280003F0C1FC2B88B02B0ED12379122B24
:107E400009D12300FA331B78012B06D10121608868
:107E500000F0E0F801E01B2BF8D037BD10B5054B62
:107E60000421187000F098F8FFF74CFDFEF770FB46
:107E700010BDC046B864FF1F0020F0B50BB20F0064
:107E800087B0834234DA274B187803F0B5FC051E1F
:107E90002BD00378A02B25D103AE3100FEF7E4F8F8
:107EA000041E0BD1B378DB0724D51F4B06341B68A7
:107EB000002B03D03100688898470400A868002888
:107EC00001D003F031FC002C08D1184A039B134069
:107ED000174A934206D0B3781B2B03D00121688840
:107EE00000F098F8280003F0C7FB802000027840DB
:107EF00007B0F0BD0F4B1B68002B10D03100688815
:107F00009847041EDAD07378002BD7D1B27801A934
:107F10000A704B800C716888FDF7F6FFCEE70624E7
:107F2000F1E7C046B864FF1FB064FF1F00FFFF0009
:107F300000011200B464FF1FF7B50190FC200D0092
:107F400017001E0003F010FC04001320002C12D0B8
:107F5000B02320002370089BF4226770658026718F
:107F60000830002B08D0190003F03EFD21000198D5
:107F700003F012FD0020FEBD089903F025FDF5E792
:107F800010B5041E06D00078FD2803D803F074FC59
:107F9000FF23237010BD00000A1F93B210B5040028
:107FA0000220032B05D882400020024BD1529B189F
:107FB0009C7010BDD864FF1F0B8870B5043B040093
:107FC0000D000220032B0BD80121200000F04CFDF6
:107FD00003001420002B03D02900200000F0DEFB5A
:107FE00070BD000007B51300034A00920A0001218A
:107FF00000F02CFC0EBDC0462182001107B5019295
:1080000003220092024B0A00122100F049FC0EBD2F
:108010009F82001107B56B4601AA11800449D880E0
:1080200008780633012802D1190003F075FC07BD5A
:10803000B964FF1F0C4B10B518700023FF210B4AC9
:108040001380138193819380094A53801370517276
:1080500093819372D174D3821375517703F08CFDA1
:1080600000F0FCF910BDC046E864FF1FD864FF1F94
:10807000BA64FF1FF0B58DB06B46002003910C224F
:108080009B5E834200DBB0E05D4B187803F0B4FBED
:10809000051E00D1A4E00378902B00D09DE006AF30
:1080A00001004688380000F013FA796804000029BE
:1080B00000D19CE03B88052B6ED13B89032B1CD95A
:1080C00005AC200000F0A2F86288172A61D839892F
:1080D000131D994231D17968237804310291D9076F
:1080E00038D5607800F08EF9071E06D000230371A2
:1080F0002378012B08D0132B23D0A868002800D1A7
:1081000078E003F011FB75E06288029909A800F09D
:10811000A6F80290380000F08BF909AA2378387A83
:108120000192002231000092029A00F012F9380008
:1081300000F064F9029B002BDFD0300000F080F9E2
:10814000DBE70378032BD8D16288029909A800F0F5
:10815000D6F8DEE7122B13D1029909A800F0B5F882
:10816000021EEAD127498B88002BC6D0887909A93D
:108170002378019161780091310000F0EAF8BCE7C2
:10818000002302AA93833000617809AAFFF72AFF2F
:10819000B3E71D4B0993F6E7042B02D09A1F012A7F
:1081A000ABD8184A043B9B00995A0029A5D0D21895
:1081B000907831003A0000F0AEF800289DD13B885D
:1081C000042B03D001213000FFF724FF012C04D140
:1081D000A868002801D003F0A7FA280003F04CFAA1
:1081E0008020039B0002434018000DB0F0BD012821
:1081F00000D182E701213000FFF70CFFEDE7C04618
:10820000E864FF1FD864FF1F010017000B7803709C
:108210004B784370CB788A781B02134343807047B6
:108220000A88030002700A88120A42700A88012A2A
:1082300006D14A8882704A88120AC27004207047A8
:1082400002208242FBD14A8804309A704A88120A7E
:10825000DA708A881A718A88120A5A71EFE710B5A3
:108260000400012082420CD94B780A781B02134388
:108270002380834206D1CB788A781B021343638024
:10828000002010BD022BFBD1CB788A781B02134350
:1082900063804B790A791B021343A380F0E70B88B4
:1082A00003700B881B0A43704B8883704B881B0A32
:1082B000C3708B8803718B881B0A4371CB888371D1
:1082C000CB881B0AC3710820704703000120082ACD
:1082D00014D14A780878120202431A80CA78887842
:1082E000120202435A804A790879120202439A80A4
:1082F000CA798879120202430020DA80704710B5EB
:1083000004000120022A05D100204B780A781B02C4
:108310001343238010BDF8B5060010200F00150090
:1083200003F022FA04000120002C0ED0A0230C221E
:10833000290023806780201D002D07D003F054FB07
:108340002100300003F028FB0020F8BD03F03CFBC7
:10835000F6E7F7B51E00009008AB142017001D7853
:10836000019103F001FA041E12D0A2230370019BB5
:1083700047704380099B057146710C220830002B21
:1083800007D0190003F030FB2100009803F004FB34
:10839000F7BD099903F018FBF6E737B5041E0FD0B7
:1083A0004388002B0CD00025C1881323007A1722A4
:1083B00001950095FFF7CDFFFF236580637225705F
:1083C00037BD000010B50C4904004A88002A09D0C6
:1083D0008B89002B05D00020CB8A0222834201D05A
:1083E00010BD012213000A20434300204032C8542C
:1083F000C81842800472F3E7BA64FF1F0023438069
:1084000003707047094B00211A0010B55C88002CDE
:1084100006D01C79844203D10A234B43D01810BDE7
:1084200001310A330329F1D10020F8E7BA64FF1FB4
:1084300010B50400407A03F01FFAFF23637210BDE9
:108440007047043010B580B203F046FB002803D01B
:108450000421494203F0B8F910BD000070B50025B1
:10846000104CA0682580A581A580A84202D003F009
:108470005BF9A56000250C4C0C4B606D1D80230042
:1084800058331D70A84202D003F04EF965650025EF
:108490006068002801D003F047F9013508340A2D3F
:1084A000F6D170BD8065FF1F2465FF1F7465FF1F37
:1084B00070B5041E09D1054D2880A881A880A86840
:1084C000002802D003F030F9AC6070BD8065FF1F5A
:1084D000F0B54B8885B00193002343600A7905000D
:1084E0000F00022A00D07BE0CA88032A17D98B68C4
:1084F0005E7819783602DC78D8790E4399781B7A41
:1085000024021B020C43034353495BBA0B80331D07
:1085100093421ED1042C04D0631F022B0ED90120DC
:1085200015E0019A4D4B1201D35A002B06D0019849
:10853000FFF7BEFF4A4A1369013313610421B8688B
:108540002E812C80494203F03FF96860002005B07D
:10855000F0BD434D042C06D0631F022B0FD9EB68EE
:108560000133EB60DBE7019A3C4B1201D35A002B3D
:1085700005D00198FFF79CFF2B6901332B61374B26
:1085800030000293019B029A1B0101930023019981
:108590008C468B52130063449C8003939E81FFF7AB
:1085A00050FF039B041E986016D00421B86849420E
:1085B00003F00AF9FA880100043A200003F014FAE3
:1085C0000199029AFB888A5A043B9B18029A8B52A3
:1085D0002B6801332B60A2E7AB690133AB619EE7E7
:1085E0001E4B0293019B1E01029BF35A002B2DD0C0
:1085F00002998C19A068002828D0012A26D1FA886F
:108600009B189BB27352A189994217D39B1AC01829
:10861000B96803F0E9F9029BA289F35A934200D0AA
:108620007DE700222B81A3882B80A3686B60029BCF
:10863000F2520B4A53680133536070E7084A93685B
:10864000013393600198FFF733FF68E7044A5369E9
:1086500001335361F6E7C046EA64FF1F8065FF1FE0
:10866000F064FF1F70B5051E15D10B4C0B4B188025
:10867000230058331870606D002802D003F054F8BE
:108680006565250050356068002801D003F04CF87E
:108690000834AC42F7D170BD2465FF1F7465FF1F1D
:1086A000F0B51700A12285B0920001934243394BE7
:1086B00006001B680C009B18D933FF331D78FDF7AB
:1086C00041FF0430854204DD3000FDF73BFF0430FC
:1086D000C5B2BD4207D33A0000213000019B03F030
:1086E0003BF905B0F0BD2900380003F04DF8230038
:1086F000C6B250331E700393019B29006365380096
:1087000003F09AF8CBB20293002B02D0039B013600
:108710001E7000262300503303931B78B34204D805
:10872000606D002831D10020DBE7029A2800002A82
:1087300004D0013B1000B34200D02800F700E71935
:10874000387003F061FA786000280ED03A78019909
:1087500003F04AF9019A3B780136D3180E4A019387
:10876000D369F6B20133D361D4E7039B1870606517
:10877000A74205D1084A1320D36A0133D362B0E778
:10878000606802F0D1FF0834F2E702F0CDFF002369
:108790006365C8E73409FF1FF064FF1FF7B50D00DC
:1087A00007000421686803F00FF82B8904000370A8
:1087B0002B891B0A43702B8883702B881B0AC3707C
:1087C0002E8902250436F6B2F42E15D81B4B9F4293
:1087D00014D10C2002F0C8FF1135011E0CD09023DB
:1087E00003708E3B0371043B4380154B8460C6804D
:1087F000187803F0D1F800252800FEBD5C237B43E8
:10880000104AD3180093583301931B78002B0FD1D3
:108810000300320038000099FFF742FF019B05007A
:108820001B78002BE8D13800009903F065F8E3E7E6
:10883000054A0725536A01335362DDE7FEFF000056
:10884000E864FF1F2465FF1FF064FF1FF0B587B0C9
:10885000009017200F0016000193FFF7F2FD13257B
:10886000041E19D00C98031E02D00199201D9847B0
:10887000030AE370052302AAA070043090812770D8
:108880000098667003A993800494FFF787FF051E84
:1088900002D0200002F048FF280007B0F0BD000021
:1088A000F0B587B01F000CAB1B7803910593012135
:1088B0000DAB06001C78049200F0D6F814250028B1
:1088C00021D02000FFF77EFD0135041E1BD0114989
:1088D000059B0A7803700132D2B2131EC68001D103
:1088E00001231A000B7022713000049B039900973A
:1088F000FFF7ACFF051E09D1230021000648074AF7
:10890000093303F089F8280007B0F0BD0023638025
:108910002370F8E7EC64FF1F9B83001130750000A3
:10892000F8B505000E00064C064F2368002B02D058
:108930003100280098470434BC42F6D1F8BDC04647
:108940009065FF1FA465FF1F0123064A5B42538009
:10895000002313715362044A136053609360D36021
:1089600013617047A465FF1F9065FF1F020000237D
:1089700010B506499C000859002801D1625010BD6D
:108980000133052BF6D11320F9E7C0469065FF1F90
:10899000034A5388181A43425841404210407047D6
:1089A000A465FF1FF0B585B002930AAB1F780CAB2E
:1089B0001B88009008000E0001920393FFF7E8FF68
:1089C00005001120002D1BD10E48FFF7E1FF040028
:1089D0001520002C14D006220B99A771E01D03F07E
:1089E00003F8019B30002371029B29006371009BF7
:1089F00066802370039B6562E381FFF791FF280087
:108A000005B0F0BDFFFF000010B5FFF7C1FF040087
:108A10000220002C12D060880121FFF781FF606ADC
:108A2000002801D002F040FE28220021200002F0A0
:108A3000CBFF012300205B426380207110BD00004A
:108A400030B5074A074C5588010013780020A5422D
:108A500004D05B1A59424B415842104030BDC046C9
:108A6000A465FF1FFFFF0000084A10B501230C009A
:108A7000904208D0FFF78CFF031E04D003792340F7
:108A80005A1E9341DBB2180010BDC046FEFF000025
:108A9000024B1879431E9841C0B27047A465FF1F6E
:108AA00070B504000D001600FFF772FF002804D116
:108AB0000D4B9C4200D0143070BD416A03790520F3
:108AC000002907D012221A40102A02D10520002EB8
:108AD000F2D10F20DB06EFD5897E0C20A942894117
:108AE000494249420840E7E7FEFF0000030010B595
:108AF000002800D110BD0348034A41889142F9D0B3
:108B00009847F7E7A465FF1FFFFF0000002330B57B
:108B1000C45CCD5C6C40D4540133102BF8D130BD13
:108B20000F23002210B5C45C64002243CA54C25C07
:108B3000D209013BF7D210BD0200010010B520326E
:108B4000103102F0A1FD10BDF0B58BB003901020E4
:108B500005931700049102F0AFFD0090102002F081
:108B6000ABFD009B13240190002B05D000280CD1F5
:108B70001324009802F098FD019B002B02D01800EE
:108B800002F092FD20000BB0F0BD102002F094FD29
:108B90000600102002F090FD13240500002E00D1E5
:108BA000AEE0002819D01022002102F00DFF3200A3
:108BB0002900039802F068FD041E0ED133787F2B44
:108BC00051D830000099FFF7ABFF009B1B787F2B3B
:108BD00053D801990098FFF7A3FF300002F064FD1D
:108BE000002D02D0280002F05FFD002CC1D1102022
:108BF00002F062FD0600102002F05EFD0290002EE1
:108C00007CD0002878D03A000F32230001251211C1
:108C100005D00F333B4015B25A4253411BB26A1E76
:108C20001201002B33D0049BD2B298180099029AFB
:108C3000FFF76CFF013D10220021300002F0C4FE5E
:108C4000ADB2049F2D017D19AF4242D0002C33D02C
:108C5000300002F029FD029B002B00D189E71800AB
:108C600002F022FD85E729003000FFF759FF2800B8
:108C70002549009AFFF74AFFA7E729000098FFF768
:108C80004FFF28002049019AFFF740FFA5E70F2179
:108C90000F4004998A18D9B28F4208D9D15C06A82E
:108CA00019540133102BF6D1029A0199C0E7791AB1
:108CB00048424141C901F2E73900300006AAFFF7F6
:108CC00025FF3200039806A902F0DEFC10370400ED
:108CD000BAE7002CBCD13000029906AAFFF716FFB4
:108CE000320006A9039802F0CFFC082204003100EC
:108CF000059802F079FEABE71324A9E71324AAE74D
:108D0000002800D06EE733E790BE0011F0B58BB0BD
:108D10000F0016000225009000283FD0002A3DD009
:108D20000B1DDBB21800029302F0C6FC1135041EC5
:108D300034D0FDF747FD05003A000099201D02F0F0
:108D4000B3FEEBB20393E3702B0CDBB22F0A00935C
:108D50006370FFB22B0E2370A7700193FDF72CFDFB
:108D60001022010006A802F09FFE2100029A04AB27
:108D700006A8FFF7E9FE051E0DD1039B08223370FC
:108D8000009B04A9B370019B7770F370301D02F053
:108D90008BFEFDF71DFD200002F086FC28000BB0C5
:108DA000F0BDF0B58FB00D00149E039004920593B2
:108DB000002A03D1022420000FB0F0BD002EF9D00C
:108DC0000398FFF7E5FD1424071EF4D0727833787A
:108DD00012021A43B3781B041343F27812061A43A3
:108DE000036A0192934201D30133E3D1002D03D0F2
:108DF0003B7901249B07DED50822002106A802F05A
:108E0000E3FD059B13240433DBB21800029302F048
:108E100053FC051ECFD0059A0499043002F044FE9D
:108E200004223100280002F03FFE390010221031E8
:108E30000AA802F039FE2900029A06AB0AA8FFF739
:108E400083FE041E0FD1082206A908A802F02CFEFA
:108E50000822311D08A802F067FE012807D10199F8
:108E60000398FDF7C9FC280002F01EFCA3E70124CB
:108E7000F9E7000070B51C4C05002368181E10D0DF
:108E8000002D14D11A78002A0CD1981C083202F057
:108E9000ABFD02F061FE0135002808D123681D708A
:108EA000012070BD0A331800082202F09DFD2368DE
:108EB000002BF5D0122002F057FC061E0DD0C12366
:108EC00021680370457002311022023002F08CFDDF
:108ED00023683100587802F05FFD206802F0E4FB5F
:108EE00000232360DCE7C046CC65FF1FF8B5040013
:108EF0002020FDF755FB0D4EA700BB590500002BA8
:108F00000DD000280BD0D878FF2809D108492A00B5
:108F10000C55F35907480333611802F07DFDF8BD85
:108F2000290002F099FD0028F0D1F8E7E865FF1F5D
:108F3000D065FF1F45A1001170B5064D840063592F
:108F4000002B05D0D87802F097FCFF226359DA7025
:108F500070BDC046E865FF1F70B506008CB00C0000
:108F6000150000213022684602F02EFD310010224B
:108F7000684602F099FD1D2021000322684402F09A
:108F800093FD6846FFF7D8FD2D2104000322280039
:108F9000694402F089FD20000CB070BDF0B50700F7
:108FA000160097B001931CAB1D7830221EAB0091C8
:108FB0000AA800211C7802F007FD102239000AA837
:108FC00002F072FD1022002102A802F0FDFC07222F
:108FD000310002A802F068FD072202AB9818631E58
:108FE0009C41019902F060FD02AB9C732B005A1E5C
:108FF000934102AAD3730021102206A802F0E4FCD8
:1090000006221D9907A802F04FFD1A2002ABC018D6
:1090100006221F9902F048FD102200990EA802F0C6
:1090200043FD102202AB0EA908781C78013A60407B
:10903000D2B2087001330131002AF5D10AA8FFF736
:109040007BFD102212A904000EA802F0CDFC102214
:1090500006AB0EA908781D78013A6840D2B20870B4
:1090600001330131002AF5D10AA8FFF765FD044359
:1090700010222098E4B212A902F016FD200017B0C9
:10908000F0BD70B50E0014008CB0010010226846CF
:109090001D0002F009FD3100082204A802F004FDC1
:1090A0002100082206A802F0FFFC6846FFF744FDF5
:1090B00004001022280008A902F0F6FC20000CB0E1
:1090C00070BDF8B506000D0000243719AC4200D37E
:1090D000F8BD02F051FB030A3B70631CDBB20137A1
:1090E0009D4203D90234F054E4B2EEE71C00EDE7F0
:1090F00073B506000C000225002819D0002917D0EE
:10910000032101A8FFF7DDFF6B469A793F231A4040
:10911000013313436A463000937101A92200FFF71F
:109120001BFF051E04D10322E01C01A902F05CFC18
:10913000280076BD03785807DA08C00FD2008000F7
:109140009B0710439B0F1843C0B2704707230B4087
:10915000C908C9000B4303707047000070B50400D4
:10916000FFF7EAFE134DA4006359002B21D0186AC3
:10917000002801D002F098FA2B59986E002801D0EF
:1091800002F092FA2B59D86E002801D002F08CFA26
:109190002B59186F002801D002F086FA2B59586F0E
:1091A000002801D002F080FA285902F07DFA00234D
:1091B0002B5170BDE865FF1F0E4B8000C35870B582
:1091C0000C00002B0FD09D68002D0CD02B78201D9B
:1091D0000B706B784B70A97CFFF7B8FF2B7E237266
:1091E0006B69E36070BD10220021200002F0ECFBEF
:1091F000F8E7C046E865FF1F014B18607047C0469E
:10920000E465FF1F074A03008000825810B5002A5A
:1092100006D0D088984203D1012901D1FFF79EFFE3
:1092200010BDC046E865FF1FF0B5264E95B087001B
:109230000B93BB590500099112200A92002B31D0E3
:10924000D888FFF7A5FB04001420002C2AD02800A2
:1092500010A9FFF7B1FFBB591E781D6A002E23D05D
:109260000895FDF7EFFA07000020FDF7F1FA0790E7
:10927000A379E61D069310AD0CA9089800F0E2FA58
:109280000EA9280000F0D7FA0B9B0A990493069BBD
:1092900009980293079B0396019300970EAB0CAAC3
:1092A000FFF77CFE15B0F0BDFDF7CCFA069030005C
:1092B000FDF7CEFAE31DA779079310AB06000893DC
:1092C000DAE7C046E865FF1F30B50C4C85002A5927
:1092D000030085B00120002A0ED018006946FFF770
:1092E0006BFF2B591A78D888054B002A00D1054B03
:1092F0006A46072100F0D9FB05B030BDE865FF1FC5
:10930000379800114598001130B5094C850029594E
:1093100085B010226846253102F066FB2A591121DA
:10932000044BD0886A4600F0C0FB05B030BDC04693
:10933000E865FF1FE198001130B5094C85002959F7
:1093400085B010226846353102F04EFB2A591121B2
:10935000044BD0886A4600F0A8FB05B030BDC0467B
:10936000E865FF1F1F990011F7B54D4F86001020CB
:10937000F4590D0002F0A0F9F3592062186A132283
:1093800000286CD0033A29009C6802F02DFBF359A9
:109390001A780192002A58D11E6A227D317B9446A8
:1093A00051400122019F114201D167461740217DA2
:1093B000914339432175377B4F40BC4660460027B7
:1093C000800701D44F081740012102208F40227DE1
:1093D00082433A432275377B5740BC46604600279C
:1093E000400701D497080F400420227DBF0082432C
:1093F0003A432275627D002794466046727B424064
:109400000A4201D167460F400121627D8A433A43F7
:109410006275777B5740BC4660460027800701D4C1
:1094200057080F400220627D7F0082431743677513
:10943000767B00227E40760701D4BA080A400426D3
:10944000617D9200B1430A4362756A78002A08D0B0
:109450006278002A05D005220533DA770022100051
:10946000FEBD04222979114205D1A17C114202D10D
:109470000533033AF1E7019A21782C78002A02D1CA
:109480000A002100140018220429E8D8042CE6D888
:1094900005206043034A05331218525CDDE7C046DD
:1094A000E865FF1FA0BE001110B50A001121024B94
:1094B00000F0FBFA10BDC0467B9900110B0030B5DF
:1094C00087B001AD2B806B4604001100981D082267
:1094D00002F08AFA2A000B212000024B00F0E5FA84
:1094E00007B030BDA399001110B50A001121024B3D
:1094F00000F0DBFA10BDC046F799001113B50B0060
:1095000011006A4613706B4604000622581C02F0D4
:109510006BFA6A4608212000014B00F0C6FA13BD21
:10952000179A001110B50A001121024B00F0BDFA84
:1095300010BDC046679A00117FB505000B4BAA000D
:10954000D4580800002C0FD0666F237FE288217862
:109550000396266F0296E66E0196A46E0094FDF7C0
:1095600009FC2800FFF7FAFD7FBDC046E865FF1F34
:1095700010B51721FFF7E0FF10BD000070B50A001D
:109580000D00064B0221040000F08FFA0600297836
:109590002000FFF7D1FF300070BDC0464799001191
:1095A00070B586B000236A461370836804001D7886
:1095B000681E0A2859D801A902F0EEFA06063337C8
:1095C0003B3F43474B4F5300180000F042F906233E
:1095D00012284BD000281BD16088FFF7D9F9082347
:1095E000002813D04279002A47D1264B1A78072346
:1095F00012070BD5244B1A680723002A06D01668D9
:10960000002E03D0290001AAB04703006A46137058
:109610006B461B786088002B2AD1FFF767FC06B0E9
:1096200070BD180000F06CF9D4E7180000F087F95D
:10963000D0E7180000F093F9CCE7180000F0ADF97E
:10964000C8E7180000F0C3F9C4E7180000F0F6F905
:10965000C0E7180000F0F6F9BCE7180000F013FAB4
:10966000B8E7180000F013FAB4E707236A4613704E
:1096700069466088FFF782FFD1E70523012AC5D13B
:10968000024BB8E77564FF1FE065FF1FE465FF1F2D
:10969000F8B52C4F8600F35904000D00002B40D084
:1096A000DA8882423DD15A78062A33D11A78002AC4
:1096B0002ED0012099681A6A097D014206D0157BD7
:1096C000054203D007225A700120F8BD0220014252
:1096D00004D0157B054201D00922F4E704200142A1
:1096E00004D0127B024201D00B22ECE7164B1B6820
:1096F000002BE9D05B68002BE6D020009847BB59CF
:1097000000215B78122BDFD12000FFF715FFDBE78C
:109710000E4BECE7112A04D1002900D03225290094
:10972000F2E7002D08D12000FFF732F9002803D01E
:10973000102302791343037121002800FDF798FAE2
:10974000C2E7C046E865FF1FE065FF1FE465FF1F35
:1097500070B50E4E8500AB590400002B13D01B785A
:10976000002B11D10A4B1B68002B04D05B68002B27
:1097700001D02000984773595B78122B03D1002148
:109780002000FFF7D9FE70BD024BECE7E865FF1F34
:10979000E465FF1FE065FF1F094B8000C3581020E0
:1097A000002B0CD01A6A002A09D09B68002B06D027
:1097B000127A1B7E101C9A4200D9181CC0B2704746
:1097C000E865FF1F70B503000D0014000220002A99
:1097D00030D000292ED013700B78081D53704B78B1
:1097E0009370FFF7A7FCE070012002212B7A237110
:1097F0006B7B034063716A7B0A40134304226371ED
:109800006E7B1640334363716E7BF608F60033437C
:1098100063712B7B0340A371287B014000200B4325
:10982000A371297B0A401343A3712A7BD208D2007B
:109830001343A37170BD10B50A0001000120FFF7AA
:10984000C1FF10BD10B50A0001000220FFF7BAFFEA
:1098500010BD70B506000C000220002E30D000298B
:109860002ED07378201D0B70B3784B70F178FFF712
:109870006DFC01223579257271794B100800134077
:10988000934010400343881010408000C9080343F0
:10989000C9000B436373B1794B1008001340934028
:1098A00010400343881002409200C9081343C900C6
:1098B0000B4321202373FCF773FE854201D2122053
:1098C00070BD2220257AFCF76BFE8542F7D82378FD
:1098D0001820042BF4D86378012BF1D80020EFE78F
:1098E000030010B50220002909D0002B07D0032265
:1098F000481C0A7019000D3202F076F8002010BDE5
:1099000003000222080010B5002B06D0002904D065
:109910000E32591C02F068F80022100010BD03003E
:1099200010B50220002909D0002B07D00422481CC2
:109930000A7019000C3202F057F8002010BD10B563
:10994000FFF7DEFF10BD03000220002906D0002B28
:1099500004D0052200200A701B784B70704703006A
:109960000220002B08D0002906D05B7800200B7065
:10997000013B082B00D918307047030010B50220B6
:10998000002909D0002B07D00622481C0A701900B4
:109990000A3202F029F8002010BD10B5FFF7B0FF21
:1099A00010BD02000B00022010B500290ED0002AC5
:1099B0000CD007211970118859701188090A997003
:1099C00011180822D81C02F00FF8002010BD030067
:1099D0000A00022010B5002B0CD000290AD099787B
:1099E0005878090201431180901CD91C082201F00B
:1099F000FBFF002010BD030010B50220002909D094
:109A0000002B07D00822481C0A701900921801F098
:109A1000EBFF002010BD02000B00022010B5002952
:109A20000BD0002A09D00921197011781818597023
:109A3000511C062201F0D8FF002010BD10B5FFF721
:109A40005FFF10BD02000B00022010B5002A09D0F4
:109A5000002907D05178197011180622581C01F0FE
:109A6000C3FF002010BD030010B50220002909D05B
:109A7000002B07D00A22481C0A701900063201F098
:109A8000B3FF002010BD10B5FFF73AFF10BD020074
:109A90000B00022010B5002A06D0002904D01800BF
:109AA0005178FFF753FB002010BDF0B585B01700CB
:109AB0001E006A4606230500080091819380FEF788
:109AC000C0FC1324011E02900CD03800B047041EC5
:109AD00005D1280001A9FEF76FFA041E02D00298F2
:109AE00001F022FE2800FFF701FA200005B0F0BDCA
:109AF000F0B504008BB0019115000021102202A8DE
:109B000001F062FF334EA700B85900283CD0C3884B
:109B1000A34239D10378002B36D14278062A18D1D6
:109B200002000100553235310C3006ABFFF7A9FABF
:109B3000002829D12000FFF72FFE020006A902A865
:109B400001F052FF200002A901F0E6FD01200BB058
:109B5000F0BD816E002917D00B8A112A28D19D42B1
:109B60000ED101981231093A01F0DEFF012807D128
:109B7000BB5920009D6EFFF70FFE29000200DEE7B3
:109B800032212000FFF7D8FC2000FEF701FF061E5F
:109B90001BD0416A002918D00B8AAB4215D108228C
:109BA0000198123101F0C0FF01280ED1716A0AE05C
:109BB0009D42E9D108220198123101F0B5FF012838
:109BC000E2D1BB59996E8A7EB9E7200001F04CFDC5
:109BD000BCE7C046E865FF1FF0B56B4D87007E59B6
:109BE00085B0337802900393002B00D087E0B368F0
:109BF000346A01937078062817D101221B7D134225
:109C000002D0217B114218D10222134202D0217BC3
:109C1000114251D10422134203D0237B134200D0BE
:109C20008BE0019B5A7DEB5991E007380428F8D866
:109C300001F0B2FF032E42678300B36E002B03D105
:109C40001C2001F039FDB066EB599C6E002C1CD035
:109C500010220021200001F0B7FE0298FFF79CFDC2
:109C600001002000FFF72DFA01F086FD2082200080
:109C700008211230FFF725FA0298FFF78DFDA07634
:109C8000EB592100D888FFF70FFC0822EB591CE0A4
:109C9000B36E002B05D01A00198AF0881232FFF734
:109CA0000DFC0222019B197DEB5911423DD0207B16
:109CB00010423AD0073208E0F488FCF7DBFD0100DF
:109CC0002000FFF711FC0A22EB595A70029B9C00FE
:109CD0002A595378073B042B11D8D088FEF758FE39
:109CE00000284ED0C3895A08D2182849029B0298EE
:109CF000CB542B5941180433254801F08DFE05B093
:109D0000F0BDFCF79FFD03000120834201D100203C
:109D10000393EB59DE88FCF79BFD039902003000AA
:109D2000FFF7ECFB019AEB59117D042211420CD094
:109D3000217B114209D00B22C7E7F688FCF73CFDD6
:109D400001003000FFF7EEFB6BE7019A527D012125
:109D50000A4204D0607B084201D00C22B5E7022100
:109D60000A4204D0607B084201D00E22ADE70421F4
:109D70000A4204D0627B0A4201D01022A5E71222D7
:109D8000A3E7FA225200B0E7E865FF1FEC65FF1F6A
:109D90004FA1001110B5064B1A780423100018408B
:109DA0001A4200D00348FFF727FA002010BDC04632
:109DB0007564FF1F2043FF1F70B50400FFF7D4FA3E
:109DC000051E43D12000FFF77FFA234EA400A059BF
:109DD0008268937CDB0708D50321036A1B790B405B
:109DE000012B02D1017F0B430377431DD97F8B1ECB
:109DF000022B0DD8022900D00121C088FCF790FF6A
:109E0000042133591A7F59700A431A77280070BD0C
:109E100001290CD102231022437000210C3001F0E3
:109E2000D3FD305910213530FFF74BF9EEE7052906
:109E3000ECD10223D118437010220C3001F0D4FD74
:109E400004233259117F0B431377EAE708251828BA
:109E5000DCD1053DDAE7C046E865FF1FF0B58BB001
:109E6000059143887E4F9E00F45915000493002C01
:109E700015D1012902D000200BB0F0BD101D57787C
:109E80001678FFF757F9EB68320002932B7A0499A2
:109E9000019300903B002000FCF70CFFEBE7E38808
:109EA000049A934201D00820E6E72378012B00D1E1
:109EB000D4E0059B581E092800D9CFE001F06CFEC4
:109EC00005CE0A29CC506C859AB229000498FFF778
:109ED00073FFD1E7200029001022453001F084FDF6
:109EE000B9594B78042B02D1013B4B70C3E70B00EF
:109EF0000A00253335320C310498FFF795F90498A0
:109F0000FFF702FA0522431E9841BB59C0005A7060
:109F1000B2E7200029001022553001F065FD049BB6
:109F20004F4C9D00295904980A0006AB55320C315C
:109F3000FFF77AF929591022453106A801F0F4FDFE
:109F4000012808D10498FFF7F7F90590002804D1FB
:109F500006222B595A7005988EE708230593FAE7D5
:109F600063780C2B7AD1E36E002B03D11C2001F017
:109F7000A3FBE066BB59D86E00286FD010222900E1
:109F800001F032FDBB590498DC6EFFF705FC0D2291
:109F9000A076BB595A706EE7E06E00285ED06378F9
:109FA0000D2B5BD12B8808220382A91C123001F0F3
:109FB0001BFDBB599A68517D0222114226D0186AB6
:109FC000407B104222D00C32E4E763780E2B45D15F
:109FD000236F002B03D1162001F06EFB2067BB59C5
:109FE000186F002803D01022290001F0FDFC0F2279
:109FF000BB59CFE763780F2B30D1206F0622691C45
:10A00000103001F0F1FCBB599A68517D04221142D5
:10A0100003D0196A497B1142D5D100210498FFF77A
:10A020008BFA28E7636F002B0DD0BB59586F0028BF
:10A03000F3D01022290001F0D7FC0122BB59524273
:10A040005B6F1A61E9E7142001F036FBBB596067CA
:10A050005B6F002BE9D126E72978DFE707200BE7C4
:10A06000E865FF1F10B5064C207001F07DFD06214C
:10A070002078FDF791FF0348FEF778FC10BDC0463D
:10A08000FB65FF1F0592001100200BB270B50D009B
:10A09000834216DA264B187801F0AEFB041E0DD071
:10A0A0000378922B0ED0A02B37D0224B1878FF28A4
:10A0B0003AD0210001F070FC002835D18020000248
:10A0C000684070BD43780E2B0BD03E2BEDD18378CA
:10A0D000052B12D0082BE8D181798088FFF7D8FAB8
:10A0E00008E0154B82889A42DFD183681878591CA2
:10A0F000FEF7C0FE002817D1D7E7104B1B785B078F
:10A1000012D50F4B1B68002B0ED09B68002B0BD079
:10A11000C289811D80889847ECE7FFF741FAA06863
:10A12000002801D001F000FB200001F0A5FAC5E7EE
:10A13000FB65FF1F1943FF1F182000007564FF1FF8
:10A14000E465FF1F10B50078FFF712FA10BD10B5D7
:10A150000078FFF7FDFA10BD0C234343084A10B501
:10A160009B185A68002A03D0012901D1904710BDDD
:10A170009B68002BFBD00029F9D19847F7E7C04630
:10A180001866FF1F01238340094A10B5946B1C43D6
:10A190009463506B98435063D46B2000984301291B
:10A1A00001D120001843D063116B0B43136310BD22
:10A1B00000800040F0B500240127154B85B0DA6B14
:10A1C000144E03921A6C0192DA64019BE3403B4205
:10A1D00017D0039DE5403D400295E5B20299280065
:10A1E000FFF7BAFF316A736A002908D03900002BE3
:10A1F00001D0029979402800FFF7C4FF01E0002B4D
:10A20000F9D101340C36172CDFD105B0F0BDC046B2
:10A2100000800040FC65FF1F064B01215A68C240C8
:10A220000A4204D01B68C3401800084070471B6DE9
:10A23000F9E7C046008000400122064B8240002919
:10A2400003D0D9680A43DA607047D9689143D9606E
:10A25000FAE7C0460038004030B5032444430F4BB2
:10A26000E25C1B199C785D7801232D1B0135AB4006
:10A27000013BA340A140DB430C00122807D808494A
:10A2800092005218116819402143116030BD054AEF
:10A2900011680B4023431360F8E7C046E7BE001186
:10A2A00008F0004014F00040C21F70B5D4B206237D
:10A2B000092C0BD80125084C9540002908D0002115
:10A2C000FFF7CAFF23682B4323600023180070BDEB
:10A2D0002368AB43F8E7C04600380040214BF0B597
:10A2E0001B185B78022B21D1032444431E4A1F4EC6
:10A2F000A35C12199478012215008540B76B013CCC
:10A30000E4B23D43A240B563194C122815D89B0016
:10A3100000290CD117495B1899680A439A600123F8
:10A32000205C154A834011680B431360F0BD11494E
:10A330005B18996891439960F1E70E4B00290DD1A4
:10A3400059690A435A61225C1328E8D00123203A54
:10A3500093400A49086803430B60E7E75969914352
:10A360005961F0E7FC65FF1FE7BE00110080004067
:10A370002CBF001100F00040A0F00040A4F000400D
:10A38000F8B500241B4E1C4D1C4B1B5D012B1FD12F
:10A39000194A9269E2401A420BD00122B256934008
:10A3A0002200143AD2B2022A09D815494A69134345
:10A3B0004B61013402360C35172CE5D1F8BD002273
:10A3C000B2560F499200521891680B439360F0E720
:10A3D000022BEED1E7B23800FFF71EFF01235840F1
:10A3E000C1B23800FFF77AFF3800FFF715FF687732
:10A3F000DFE7C046B9BE0011FC65FF1FFD65FF1F0A
:10A4000000F00040012202388240054B002903D0B1
:10A4100059690A435A617047596991435961FAE78A
:10A4200000380040F8B50E0001210F008740114AA6
:10A430000400D368FD43BB43D360831E8B4201D825
:10A44000FFF7E0FF00212000FFF72EFF0A4A0B4B29
:10A450005168012E05D139431B1951605E700020EF
:10A46000F8BD2940516002221C1962709A6915409A
:10A470009D61F4E70038004000800040FC65FF1F4C
:10A48000012210B58240074B002906D019680A4303
:10A490001A600121FFF7C6FF10BD196891431960CA
:10A4A000F7E7C046008000400C2370B50025434309
:10A4B0000A4A29009B181D70094B04001B185D7087
:10A4C000FFF7B0FF0123A340064928000A681A439A
:10A4D0000A6005490A689A430A6070BD1866FF1F42
:10A4E000FC65FF1F348000403080004070B50400E0
:10A4F0000E00FF2813D003250540FFF7D5FF084ABB
:10A50000A3089B009B183F22ED00AA40AE401968AB
:10A5100020009143314319600121FFF78DFE70BD8A
:10A5200018380040F8B50C244443134B0500E418D8
:10A530006368002B03D1A3681220002B1AD00222DB
:10A5400001270E4B00215B195A7028002770FFF776
:10A5500069FF63681E1E08D0A3683E00002B04D06C
:10A560002800FFF759FE4640F6B228003100FFF7F9
:10A5700009FE0020F8BDC0461866FF1FFC65FF1FDE
:10A58000F7B5C420FF222B4B8000195800249143BB
:10A590003F3A0A431A508022274F5202274E1A6030
:10A5A000274B1D5D002D21D0A31E012B03D80121B7
:10A5B000E0B2FFF727FF012D18D11F4B9B69E34045
:10A5C0002B4213D0E3B218000193FFF725FE0100E0
:10A5D0000198FFF755FFE3B2143B022B1DD8012170
:10A5E0007156184A8D405369AB4353613B7F002B32
:10A5F0000DD0E5B22800FFF795FF2800FFF70CFE0D
:10A600007B7F0100834202D02800FFF7A5FD0134C3
:10A610000C370236172CC3D1F7BD01210023715628
:10A62000F3568D40074A9B009B189A68AA439A608C
:10A63000DCE7C04600E100E0FC65FF1FB9BE001189
:10A64000FD65FF1F00F0004070B50E00150004000E
:10A65000FFF72AFF0C236343094A20009B189D60E3
:10A660005E60FFF75FFFF021064B074A8900051E79
:10A670005A5002D02000FFF717FF280070BDC046D7
:10A680001866FF1F0000FF1FB5A1001170B5134D24
:10A6900007202C78002C1FD198222100520028007E
:10A6A00001F09AFA0123C420FF222B700C4B80008A
:10A6B0001C635C630B4B1C605C600B4B1958914333
:10A6C0003F3A0A431A50802252021A600D20074A6C
:10A6D000074900F0A1FF200070BDC046FC65FF1FC8
:10A6E00000800040A0F0004000E100E081A50011E2
:10A6F00081A30011030010B50620072B09D8054AD5
:10A70000137001F079FAD7210020034B034A890026
:10A710005A5010BD4843FF1F0000FF1F911BFF1F31
:10A7200070B51D0002240C2910D8094ACA40D2076E
:10A730000CD5FBF741FF041E08D1059A04992800A7
:10A74000FBF756FFFCF7C4FDFFF724FB200070BDAC
:10A750001210000030B50D7802232C009C431842E3
:10A7600001D02B431C0008252300AB43284201D015
:10A770002B00234320241D00A543204201D01C436D
:10A7800025002A230D70184204D011781E3B0B437C
:10A79000137030BD0028FCD10C2113788B43F7E7F0
:10A7A000F8B51D0006AB1B88140007AA0E000B208D
:10A7B0001778002B27D10A78022A49D14A685078A5
:10A7C00011780002244A08438018042840D801F078
:10A7D000E3F903121D1B2300F06800F05DFF021C6B
:10A7E000C0B2B84200D93A1CD2B22000F1682A8027
:10A7F00001F0FAF806E00222F3681B882A80237031
:10A800001B0A63700020F8BD0622EEE701232B80AF
:10A81000F3681B782370F5E7F368002B16D0082245
:10A820002A801A8822701A88120A62705A88A270C6
:10A830005A88120AE2709A8822719A88120A627102
:10A84000DA88A271DB881B0AE371DBE72B80D9E78A
:10A8500001202B80D7E7C04600D6FFFFF7B51600D2
:10A860000A781D0008AB1F880C000123022A18D1AA
:10A870004A685078117800022B4A08438018032850
:10A880000FD801F089F902254439E06800F004FF8F
:10A89000C0B20723B84204D37B190193152B02DD04
:10A8A0000D231800FEBDE0682A003100C01901F038
:10A8B0009BF86B4600209B88E268D0541B4B1B68BA
:10A8C000834203D01B68834200D098470023E8E707
:10A8D0000B23002FE5D1022DE2D1737832781B02D1
:10A8E0001343E2681380114B1B68002BEED01B68EA
:10A8F000002BEBD00120E8E70B23002FD1D1062D50
:10A90000CED12A003100E06801F06EF8DEE70B23BB
:10A91000002FC6D1012DC3D132787533012AC0D89A
:10A92000E3681A70D2E7C04600D6FFFF0868FF1F31
:10A9300070B50C001500072837D801F02DF9041464
:10A9400036361B36242E182015290BD8184E162201
:10A950000021300001F038F822002900300001F019
:10A9600043F8002070BD18200229FBD11288114B3A
:10A970001A80F6E718200829F4D10A000E482900A9
:10A9800000F01AFFEDE718200129EBD10B4B1078EE
:10A990000B49DA69FFF7DEFEE3E718200129E1D170
:10A9A000064B10780749DA6BF4E70220DAE7C04675
:10A9B000F067FF1FC643FF1FBC43FF1F4C43FF1F31
:10A9C0007443FF1F9443FF1F030010B50020DB07F3
:10A9D00004D50721024A034800F08CF810BDC04698
:10A9E00044BF00114C43FF1F054A030010680028B4
:10A9F00003D082889A4201D1806870470068F6E7E8
:10AA0000006AFF1F0A88030008009A4204D08A885F
:10AA100004309A4200D0002070470000F8B5F222BE
:10AA200000230D4F0D4E7968050042433370994263
:10AA300000D07B600A4C0021200000F0C5FF0023FD
:10AA40001A007C60AB4202D100203370F8BD0133A4
:10AA50002280DBB2F234F5E7F86AFF1FF66AFF1FC7
:10AA6000046AFF1F73B56B46019006006846150027
:10AA70001980FCF75FFF041E11D1002D0FD07689DD
:10AA8000002E11D00C2000F017FE00280ED0084A2E
:10AA90000460136886808560002B02D1106020005E
:10AAA00076BD1A001B68F7E70224F8E71324F6E7DF
:10AAB000006AFF1F012100220A4B10B549420A4CCF
:10AAC000198099809A719A70084B20700120198022
:10AAD0005A60FFF7A3FF2078FCF78AFF0448FDF7D0
:10AAE00045FF10BD1068FF1F006BFF1FF86AFF1FB6
:10AAF000A1AB0011022310B5002802D0FFF7B2FF6E
:10AB00000300180010BD0000030010B50020DB0793
:10AB100004D50421024A0348FFF7A4FF10BDC04634
:10AB200058BF0011CC43FF1FF0B50E2687B003932A
:10AB30000CAB1F8802ABF61805000800310002922A
:10AB4000FDF77AF804000120002C0FD03088FFF7C1
:10AB50004BFF03000E20002B08D05E68002E05D0AE
:10AB600021002800039B029A0097B04707B0F0BD70
:10AB70000A4B10B5984207D10122002352420A80A5
:10AB80008B708A808B7110BDFFF73CFF0028FAD0D4
:10AB900001235B42038000238370F4E7FFFF000082
:10ABA000F8B5050001290AD1134E00243388F22795
:10ABB000AB4219D028001149FFF7DAFF06E002295D
:10ABC00004D10139FDF750FF0028EDD0F8BD3B005E
:10ABD00063437268D018D35A002B09D03A00002181
:10ABE00000F0F2FE0134E4B2054B1B78A342EED82C
:10ABF00001235B423380DDE7F86AFF1F1068FF1F07
:10AC0000F66AFF1F10B5FFF7FDFE03000020834228
:10AC100000D0987810BD0000F0B589B01C000EABD4
:10AC200080CB03901E8810AB1B78049202930B7AA2
:10AC30000D00DB0616D42B780593022B24D0049844
:10AC4000FFF7D2FE002812D003689C46002B0ED0DE
:10AC5000029B2200019329003B0064460398009662
:10AC6000A04705E00498FFF7BFFE002802D10E20A0
:10AC700009B0F0BD8368002BF9D00A22290003989F
:10AC800098470028D7D0F3E76B6858781A786B4B51
:10AC9000000210439842D2D8043B984210D2684B2D
:10ACA000984242D015D8674BC0180128C7D80B204E
:10ACB000002EDDD1EB681A7859683A80200028E030
:10ACC000614BC018032800D979E000F065FF846A61
:10ACD000789E5E4B9842B2D10B20002EC8D1012342
:10ACE0003B80EB6831001B7823706889013080B2AB
:10ACF000FCF7A2FF3A88031E0ED0017802328A18B0
:10AD00003A80428962704289120AA27059680278B8
:10AD1000E01C00F069FE06E004323A8031000422B3
:10AD2000601C00F051FE0020A2E70B20002E9FD1F6
:10AD3000EB6807A91E8804233B80330A3000267085
:10AD40006370FCF779FF051E28D004AB9A890E23A7
:10AD500004A95B183E49C668FCF7E2FF00280BD146
:10AD60002B783C486A680599FBF798FB002803D1CB
:10AD7000012304AA5B42D3813278022A06D171688A
:10AD8000201D00F031FE3B8802333B800E2304AAD5
:10AD90009B181B88A3701B0AE370C4E704ABDE8119
:10ADA000F4E70B20002E00D062E7E9680398FFF774
:10ADB00029FF02233B802070000A6070B3E70B205C
:10ADC000002E00D054E70222EB681B883A802370E3
:10ADD0001B0A6370A7E7E86800F05EFCC2B20300DC
:10ADE0000720B24200D243E70DD00299DBB27118BE
:10ADF000994202DB921BD3B20293029BE9681A00CC
:10AE00003B8089195AE70023F6E70B20002E00D07B
:10AE10002EE70722EB683A801A7822705A7862701F
:10AE20005A88A2705A88120AE2701A792271DA8856
:10AE30006271DB881B0AA37175E7C0460429000014
:10AE40000228000000D8FFFFFFD6FFFF0328000004
:10AE5000FFFF000088BE0011F0B58DB06B460020EA
:10AE6000089120229B5E83423DDAA64B187800F0C1
:10AE7000C3FC071E32D00378B02B2CD100790238E6
:10AE800016281FD800F0E0FD17001E001E001E004F
:10AE900031001E0096001E001D011E0052011E0002
:10AEA00073011E00CD011E0050021E001E001E0078
:10AEB0008E021E00E302944B94491B8878880B8015
:10AEC000FBF72CF83800FCF7ADFF914B1B68002B0B
:10AED00001D038009847380000F0CEFB8020089B56
:10AEE0000002434018000DB0F0BDEE22002187485B
:10AEF00000F06AFD0BAA3B7B7989388900923A0001
:10AF00000D32FCF7B1FD0400804B1B78002C3FD1C3
:10AF100046E0804B788805937F4B4100CB5A0BAEBF
:10AF2000073BDBB232880293002301937B4B210065
:10AF300006930093059BFFF76FFE744D002810D118
:10AF4000069B3A8A1B889A420BD138000599123029
:10AF500000F0EAFD002804D02B7862899B00EB18F2
:10AF60005A80162306A81B18328820007989FCF71E
:10AF7000D7FE2B7804009A00AA1851880029C3D064
:10AF80000133DBB22B70002807D006A9C98A918053
:10AF9000634A12889A42BCD802E00121494291805A
:10AFA000002B04D059497888FAF7ECFF8AE73E89EC
:10AFB0000A2479E000253E89574B06937B88069A40
:10AFC0005B009B5A033B9D4202DB002DF0D05BE00F
:10AFD000162206A812183B7B798900923A003000AD
:10AFE0000D32FCF741FD0590002858D04689017AC2
:10AFF0007888FCF703FD041E44D1464B78880793FC
:10B00000069B4100C95A454B0439C9B206AAD28AE7
:10B0100006930291019400930599079BFFF7FCFDAD
:10B02000041E2FD1069B39491A88931C002D26D166
:10B030004B807988384B4900CB5A5119033B8B42DE
:10B0400020DD059B31485B8941190B71A91C013535
:10B05000C9B2EDB2059145191B0A2B71059B2D490B
:10B060000433181800F0C0FC2C4B059A1B88D31829
:10B07000DDB22C4B9E4205D00136B6B29CE7498822
:10B080009942D6D0002D0CD0204C2800618800F0C9
:10B090006BFC207021007888FAF784FF12E7059C8A
:10B0A000F0E7002C00D183E77B78142B00D109E76F
:10B0B00016493B794E800B700C717888FAF724FFA3
:10B0C00000E7162406ABE41821003889FCF7B4FD2C
:10B0D000011E00D1B7E1788822880F4C45002C5B17
:10B0E0000A4D013CE4B2029400240F4B01940095F8
:10B0F000FFF792FD041E00D014E129007888FAF7CA
:10B1000061FFDFE6006BFF1FB842FF1F1868FF1FDB
:10B110000C68FF1F0C69FF1F4864FF1FFC69FF1FBD
:10B12000B642FF1FFFFF00001A68FF1F162406AB80
:10B13000E41821003889FCF77FFD011E00D182E16F
:10B1400078882288AE4C45002C5BAE4D013CE4B2C1
:10B1500002947C89AC4B01940095FFF75DFD041EC1
:10B1600000D0DFE029007888FAF736FFAAE600254C
:10B17000A44B1D803B00F6331B78A24A78880792C7
:10B18000AB4208D99E4B12880693069943005B5A3E
:10B19000013B9A4203DB0799FAF728FF92E616244F
:10B1A0006B00FB18059306ABE418059B210018897A
:10B1B000FCF742FD011E03D1059B01241E8973E7A4
:10B1C0007888924B2288069C099343001B5B904E23
:10B1D000013BDBB20293002300960193099BFFF72A
:10B1E0001BFD041E02D0059B1E895DE77B88069A25
:10B1F0005B009B5A079A108832881218934202DC2F
:10B200001B1A013B33807F4C0230328809990019A8
:10B2100000F0EAFB2388328801359B182380EDB2C9
:10B22000A8E70BAA3B7B7989388900923A000D3256
:10B23000FCF71AFC00250590059B002B04D10A247D
:10B24000002D00D16EE060E0059B7888197AFCF74C
:10B25000D5FB0100041E63D1694C6C4B78880694C1
:10B260000993069B4400E45A694B063CE4B20BAEDA
:10B27000328807930294019100930599099BFFF787
:10B28000CBFC041E4CD1079B5E491B881A1D002D68
:10B2900030D14A80059B5B4C5A8963191A716B1C2B
:10B2A0009BB2E318120A1A71162306A832881B18DB
:10B2B00079890598FCF734FDFF21AA1C2E1D033562
:10B2C0000B00059092B2B6B2ADB2002803D006AB27
:10B2D000DB8AD9B21B0AA218651911712B714C4D6A
:10B2E000301D2A884949201800F07EFB2B88F6186B
:10B2F000B5B2A1E74988914207D17A8806995200F0
:10B30000525AEB18053A9A42C4DC3E4C2800618838
:10B3100000F03AFA207021007888FAF771FED1E542
:10B32000002DF2D13E89BFE6162606ABF618310095
:10B330003889FCF781FC3D000400FA3500282DD047
:10B34000037A9B060CD400227B8939897888009285
:10B350003A000C32FFF7E8FB041E10D03E8915E0DE
:10B360003088FFF741FB00281AD08368002B17D0E4
:10B370002100122278889847041EE4D0EEE72B784B
:10B38000002B02D17888FAF74BFE00262B78002B91
:10B3900000D097E5002C00D194E585E60124DDE797
:10B3A0000E24DBE7162506ABED1829003889FCF7DB
:10B3B00043FC041E47D0037A9B0611D4154A7B88B0
:10B3C0001188994203D01448814207D11380134B4E
:10B3D000F2261D780023D9B2A94221D30924A1E77E
:10B3E0002888FFF701FB00282FD08368002B2CD082
:10B3F0002100122278889847041EDFD092E7C046C9
:10B400004864FF1F1868FF1F1A68FF1F0C69FF1FA1
:10B41000FC69FF1FF86AFF1FFFFF0000F66AFF1FAD
:10B4200031005943546801336018615A0029D2D160
:10B430003C0008342100F22200F0D6FA210078887E
:10B44000FAF7F6FD3EE501246CE70E246AE71D4B92
:10B450001A887B889A4231D07888FAF7F3FD31E573
:10B46000F223059851684343CD18C95A00291FD0CB
:10B470003B7A012B0BD16C88AB887888AA1D00948D
:10B48000FFF752FB041E02D000233B722E88F222EB
:10B490000021280000F098FA00232B80059B01333F
:10B4A000DBB20593084B05991B78064A8B42D7D827
:10B4B00001235B421380002CCED0F5E5002634003A
:10B4C0000596EFE7F86AFF1FF66AFF1F70B50400E4
:10B4D0000E001500FFF796FA031E08D1310005484B
:10B4E000FFF790FA03001120002B02D01C800020EF
:10B4F0009D7070BDFFFF0000F8B50B4F06003B7854
:10B500000D001400FF2B0ED00A2000F02DF9011EB3
:10B5100009D0B1230380002346800371C5800481D4
:10B52000387800F039FAF8BD0D44FF1FF7B50F0069
:10B5300008A90600088809A90B240988002821D138
:10B540000234022B1ED1557813782D021D432B0097
:10B550008B4301937334002B14D1FB683000190026
:10B560000093FFF74FFB019C85420BD02A0030006F
:10B570000099FFF7ABFF041E04D12A00300079893F
:10B58000FFF7BAFF2000FEBDF0B50E7885B003903E
:10B590000AA805880120022E0DD14C68277864780E
:10B5A00024023C43054FBC4205D10398DBB201960F
:10B5B0000095FFF7BBFF05B0F0BDC04602290000B3
:10B5C000034B10B51B68002B00D09847FEE7C04620
:10B5D000046BFF1F07B501A8FFF7F2FF044A0548F7
:10B5E0000021121A00F0F8FAF8F70CF9FEE7C0464D
:10B5F000086BFF1F1044FF1F01B40248844601BCC2
:10B60000604700BFC9A9000001B40248844601BCDC
:10B61000604700BF5522000001B40248844601BCC7
:10B62000604700BF1131FF1F01B40248844601BCCE
:10B63000604700BF156B010001B40248844601BC9D
:10B64000604700BFFD38FF1F01B40248844601BCBB
:10B65000604700BFA54F010001B40248844601BC09
:10B66000604700BF8D12000001B40248844601BC4F
:10B67000604700BF091B000001B40248844601BCBA
:10B68000604700BF434D010001B40248844601BC3D
:10B69000604700BFE548000001B40248844601BC91
:10B6A000604700BFDD52010001B40248844601BC7E
:10B6B000604700BF014C010001B40248844601BC50
:10B6C000604700BF3D4B010001B40248844601BC05
:10B6D000604700BF2124000001B40248844601BC39
:10B6E000604700BFED4A010001B40248844601BC36
:10B6F000604700BF8552010001B40248844601BC86
:10B70000604700BF9D3AFF1F01B40248844601BC58
:10B71000604700BF8B52010001B40248844601BC5F
:10B72000604700BF311B000001B40248844601BCE1
:10B73000604700BFD949010001B40248844601BCFA
:10B74000604700BF456B010001B40248844601BC5C
:10B75000604700BF056A000001B40248844601BC8E
:10B76000604700BF3539FF1F01B40248844601BC61
:10B77000604700BF1D4D010001B40248844601BC72
:10B78000604700BF2951010001B40248844601BC52
:10B79000604700BF090E000001B40248844601BCA6
:10B7A000604700BFC94A010001B40248844601BC99
:10B7B000604700BF055E000001B40248844601BC3A
:10B7C000604700BF810E000001B40248844601BCFE
:10B7D000604700BF5549010001B40248844601BCDE
:10B7E000604700BF7539FF1F01B40248844601BCA1
:10B7F000604700BF5125000001B40248844601BCE7
:10B80000604700BFF54E010001B40248844601BC08
:10B81000604700BFF30E000001B40248844601BC3B
:10B82000604700BF0934FF1F01B40248844601BCD1
:10B83000604700BF291C000001B40248844601BCD7
:10B84000604700BF090E000001B40248844601BCF5
:10B85000604700BF75A9000001B40248844601BCDE
:10B86000604700BFB352010001B40248844601BCE6
:10B87000604700BFE938FF1F01B40248844601BC9D
:10B88000604700BF1147010001B40248844601BC73
:10B89000604700BFF94C010001B40248844601BC76
:10B8A000604700BF6DBC000001B40248844601BC83
:10B8B000604700BF4550000001B40248844601BC07
:10B8C000604700BF3D18000001B40248844601BC37
:10B8D000604700BF4137FF1F01B40248844601BCE6
:10B8E000604700BFADAE000001B40248844601BC11
:10B8F000604700BFF537FF1F01B40248844601BC12
:10B90000604700BF3519FF1F01B40248844601BCDF
:10B91000604700BF4D1F000001B40248844601BCCF
:10B92000604700BFE117000001B40248844601BC33
:10B93000604700BF8930FF1F01B40248844601BC44
:10B94000604700BF7136FF1F01B40248844601BC46
:10B95000604700BF9DA9000001B40248844601BCB5
:10B96000604700BF0919FF1F01B40248844601BCAB
:10B97000604700BF350E000001B40248844601BC98
:10B98000604700BF350E000001B40248844601BC88
:10B99000604700BFB54C010001B40248844601BCB9
:10B9A000604700BF594F010001B40248844601BC02
:10B9B000604700BF5D17000001B40248844601BC27
:10B9C000604700BF2146010001B40248844601BC23
:10B9D000604700BF154D010001B40248844601BC18
:10B9E000604700BF213AFF1F01B40248844601BCF2
:10B9F000604700BFE94C010001B40248844601BC25
:10BA0000604700BF7130FF1F01B40248844601BC8B
:10BA1000604700BF691F000001B40248844601BCB2
:10BA2000604700BFA946010001B40248844601BC3A
:10BA3000604700BF312EFF1F01B40248844601BC9D
:10BA4000604700BFC51D000001B40248844601BC28
:10BA5000604700BF353BFF1F01B40248844601BC6C
:10BA6000604700BF5147010001B40248844601BC51
:10BA7000604700BF0D52010001B40248844601BC7A
:10BA8000604700BFF13AFF1F01B40248844601BC81
:10BA9000604700BF4136FF1F01B40248844601BC25
:10BAA000604700BF6571010001B40248844601BCD3
:10BAB000604700BF4551010001B40248844601BC03
:10BAC000604700BFB132FF1F01B40248844601BC89
:10BAD000604700BF0D3BFF1F01B40248844601BC14
:10BAE000604700BFE928000001B40248844601BC59
:10BAF000604700BF2526000001B40248844601BC0F
:10BB0000604700BF4D36FF1F01B40248844601BCA8
:10BB1000604700BF5952010001B40248844601BC8D
:10BB2000604700BFC56D010001B40248844601BCF6
:10BB3000604700BFCD4C010001B40248844601BCFF
:10BB4000604700BFEDA5000001B40248844601BC77
:10BB5000604700BFB539FF1F01B40248844601BCED
:10BB6000604700BFD91B000001B40248844601BCF5
:10BB7000604700BFC926000001B40248844601BCEA
:10BB8000604700BF7918000001B40248844601BC38
:10BB9000604700BFB14E000001B40248844601BCBA
:10BBA000604700BF213BFF1F01B40248844601BC2F
:10BBB000604700BF851F000001B40248844601BCF5
:10BBC000604700BFC521000001B40248844601BCA3
:10BBD000604700BF0124000001B40248844601BC54
:10BBE000604700BFB70E000001B40248844601BCA4
:10BBF000604700BFD932FF1F01B40248844601BC30
:10BC0000604700BF911BFF1F01B40248844601BC7E
:10BC1000604700BF017F000001B40248844601BCB8
:10BC2000604700BFC93AFF1F01B40248844601BC07
:10BC3000604700BFDD66010001B40248844601BCD4
:10BC4000604700BF3555000001B40248844601BC7E
:08BC5000604700BF1D4B01001D
:10BC580000030102020303030403050006020700B0
:10BC6800080209030A030B030C000D000E030F035F
:10BC7800100311031303140315021602B13B00113C
:10BC8800E53B001100000000020000009ABC001112
:10BC9800192A0F180A000000F1590000FD240000BD
:10BCA800414601007580001189A00011DD74001162
:10BCB800797E00112553001159AE0011714F001102
:10BCC800C13D0011F13E00110000000016160000F1
:10BCD80002000000E4BC0011F4FFF3FFD2FC0000F6
:10BCE8003140001100000000000000005475796127
:10BCF8000042312E3800303031370067697468757A
:10BD0800622E636F6D2F707676780054484231004A
:10BD1800020000002CBD0011292A282A272A262AD9
:10BD2800252A242A0A180000E204000071020000F3
:10BD380078EC0000050000007440000010270000A7
:10BD480060F000000400000006640000204E0000BF
:10BD58000000000006000000050000001F501D0044
:10BD6800023CB4000001170018000000A102000006
:10BD78003031323334353637383941424344454619
:10BD880000000000295700117D5700110000000035
:10BD980002000000A4BD00116F2A6E2A1A18EAD802
:10BDA800BC80F0FC600000000000000000005F069E
:10BDB8006B2F363D7D077F3F777C596E7971000088
:10BDC80001A00000000000006410B71DC8206E3BF1
:10BDD800AC30D9269041DC76F4516B6B5861B24D8A
:10BDE8003C7105502083B8ED44930FF0E8A3D6D6F4
:10BDF8008CB361CBB0C2649BD4D2D38678E20AA05C
:10BE08001CF2BDBDFB349B5F800000800010000069
:10BE180000000000DF600011697700110361001164
:10BE2800717B001187610011477B0011FD610011D2
:10BE38001D7B00114F620011E57C0011B7620011F3
:10BE4800E57C0011E96200119F7C0011FD61001181
:10BE5800D57A0011756200117D7C00110000000088
:10BE6800000000005B6300117D7C0011BD630011C0
:10BE780081770011052A042A012A002A02290328A9
:10BE88000128002801180018000000000000000028
:10BE98000000000000000087010102010201010208
:10BEA800010203030401030101010101030302016B
:10BEB80003000D000E00100011001300140107010B
:10BEC80008010A010B011C011D02040205020702F8
:10BED800080219021A021C021D03010302031700BB
:10BEE8000201000504000807000B0A001716001DD0
:10BEF8001C010201010504010E0D011110011413AA
:10BF0800011716011A19020201020B0A020E0D028C
:10BF18001110021413021716030504030807030B74
:10BF28000A030E0D0001020307090A0B0E0F101178
:10BF380012141718191A1B1F20212200A1A700117B
:10BF48005DA8001100000000020000008EBE001174
:10BF58000000000089B50011000000000200000088
:04BF68008CBE00117A
:020000041FFFDC
:1000000000000000293D0011A0BC00119CBC0011A3
:100010004061FF1F00000000000000000000000021
:1000200000000000000000000000000000000000D0
:1000300000000000000000000000000000000000C0
:1000400000000000000000000000000000000000B0
:1000500000000000000000000000000000000000A0
:100060000000000000000000000000000000000090
:100070000000000000000000000000000000000080
:100080000000000000000000000000000000000070
:100090000000000000000000000000000000000060
:1000A0000000000000000000000000000000000050
:1000B0000000000000000000000000000000000040
:1000C0000000000000000000000000000000000030
:1000D0000000000000000000000000000000000020
:1000E0000000000000000000000000000000000010
:1000F0000000000000000000000000000000000000
:1001000000000000000000000000000000000000EF
:1001100000000000000000000000000000000000DF
:1001200000000000000000000000000000000000CF
:1001300000000000000000000000000000000000BF
:1001400000000000000000000000000000000000AF
:10015000000000000000000000000000000000009F
:10016000000000000000000000000000000000008F
:10017000000000000000000000000000000000007F
:10018000000000000000000000000000000000006F
:10019000FD32FF1F5D31FF1FC1660100000000003E
:1001A000000000000000000000000000000000004F
:1001B000000000000000000000000000000000003F
:1001C000000000000000000000000000000000002F
:1001D000000000000000000000000000000000001F
:1001E000000000000000000000000000000000000F
:1001F00000000000000000000000000000000000FF
:1002000000000000000000000000000000000000EE
:1002100000000000000000000000000000000000DE
:1002200000000000000000000000000000000000CE
:1002300000000000000000000000000000000000BE
:1002400000000000000000000000000000000000AE
:10025000000000000000000000000000000000009E
:10026000000000000000000000000000000000008E
:10027000000000000000000000000000000000007E
:10028000000000000000000000000000000000006E
:10029000000000000000000000000000000000005E
:1002A000000000000000000000000000000000004E
:1002B000000000000000000000000000000000003E
:1002C000000000000000000000000000000000002E
:1002D000000000000000000000000000000000001E
:1002E000000000000000000000000000000000000E
:1002F00000000000000000000000000000000000FE
:1003000000000000000000000000000000000000ED
:1003100000000000000000000000000000000000DD
:1003200000000000000000000000000000000000CD
:1003300000000000000000000000000000000000BD
:1003400000000000000000000000000000000000AD
:10035000000000000000000000000000000000009D
:10036000000000000000000000000000000000008D
:10037000D5B50011000000000000000000000000E2
:10038000000000000000000000000000000000006D
:10039000000000000000000000000000000000005D
:1003A000000000000000000000000000111BFF1F03
:1003B000000000000000000000000000000000003D
:1003C000000000000000000000000000000000002D
:1003D000000000000000000000000000000000001D
:1003E000000000000000000000000000000000000D
:1003F00000000000000000000000000000000000FD
:08183800106FFF1F4118FF1F94
:10184000024981F3088802F0F7FA0000106FFF1FC9
:1018500070B500241E491F4A1F484C6308CA1B0567
:101860001B0DE4188242F9D11C4B80228B630021AE
:1018700009201B4B920519621A4B1B4DDA671B4B53
:10188000DA688243DA609A68194802409A60112047
:10189000296002F08FF8112002F06CF86B6C154A89
:1018A000112013406B64EE23DB006343124A1B0CD0
:1018B00013840122114B9A7201F006FC104B1B7825
:1018C000002B04D10F4B1021187802F025FA70BDBF
:1018D000000005400806054080060540FF010000A5
:1018E00000F0004004E100E0003800403CF000401F
:1018F000FFDFFFFFFFFEFFFF1061FF1FC461FF1F3F
:10190000F263FF1FF061FF1F10B502F025F90728F1
:1019100004D0122808D0022808D010BD044A0420A0
:10192000136B01331363F8E70220F6E71420F4E7A2
:10193000F064FF1FF8B507000C00260025005036A4
:1019400030785135002804D10300287058342370B2
:10195000F8BD2978CA00481E8141A3183800A25C4E
:101960005B68C9B2FFF7D0FF00280DD12B78DA00F1
:10197000A218013350602B703378044A013B337056
:10198000136A01331362D8E70123DFE7F064FF1F16
:101990005C234343074910B5C9180B0058331B7823
:1019A000012B05D1FFF7C6FF034A936A0133936207
:1019B00010BDC0462465FF1FF064FF1F10B502F084
:1019C00033FB064A0121130010CB4942D967044B6F
:1019D000136002F049F9200010BDC04600E100E0AC
:1019E0001000100010B5040002F01EFB024B1C603A
:1019F00002F03AF910BDC04600E100E0431E5A4231
:101A00005341A022F0B5D2015B421340154D164A56
:101A100040019B182A18127E8BB00191002A1BD01E
:101A20001A000832D46F0022E6B206AFE4B2944244
:101A30000EDC2818C369002B08D0019902AA117185
:101A400006AA049202AA167303A898470BB0F0BD29
:101A50001978B9540132EAE71A7D1A7806AB0126E3
:101A60001A70E6E7B067FF1F00400040F0B5254B55
:101A700004004001C25C85B0002A2BD01A18117EE8
:101A8000002927D0917E002924D01179022921D163
:101A90001689D788D168F51BADB22A1C102D00D944
:101AA000102292B2BE4217D11818012303710023ED
:101AB000C269C38003819A4206D06846032103733A
:101AC0000171029301A890470820002C00D0192032
:101AD00001F0FAFA05B0F0BD013C65426C41A02569
:101AE0006442ED012C40084D1B186419074D063364
:101AF000013A92B2AA42EDD01888461C1E80085CBA
:101B00002070F5E7B067FF1F00400040FFFF0000B6
:101B10000F220E4B10B59868104002380A280BD8D7
:101B200001F0FEFF0D0A0B0A0A110A0A0A0A060052
:101B300002210020FFF762FF10BD0121F9E700201C
:101B4000FFF794FFF8E7DB6FF6E7C0460040004080
:101B50000F220E4B10B59868104002380A280BD897
:101B600001F0DEFF0E0A0B0A0A120A0A0A0A060030
:101B700002210120FFF742FF10BD01210800F9E713
:101B80000120FFF773FFF7E7DB6FF5E700900040F8
:101B900013B5334C2378072B3DD8324B1A78324B90
:101BA000002A39D18022196852020A431A6025207E
:101BB00001F0C0FE20232D4A11680B4380211360E1
:101BC0006B460422C90508680733104228D08021DB
:101BD0000422C905C86810422ED080212020C905E2
:101BE000CA688243CA6014221A701A78002A2FD158
:101BF0008021C905C86820320243CA6014221A70C5
:101C00001A78002A28D11A4B1A7D22785A601D2290
:101C10001A705932DA6013BD1A6816490A40C5E7CE
:101C2000086802430A6014221A701A78002ACED07B
:101C30001A78013AD2B2F7E7C8680243CA601422A0
:101C40001A7019784A1ED2B21A700029F9D1C4E765
:101C50001A78013AD2B2C7E71A78013AD2B2CEE77F
:101C60004843FF1F1044FF1F3CF000404043FF1F4C
:101C700000200040FFFFFEFF564B70B51B68012B94
:101C800003D1554A936D0133936502F08DF9534B9F
:101C9000534A1860534B544C1A600123534A136043
:101CA000534A13602378002B06D00622514952482C
:101CB00001F072FF00232370504A514B10681B78CB
:101CC000C1B2002B0ED14F4CC0B223785BB2002BB7
:101CD0004FDB237824785BB264B21B0424021B1907
:101CE0001B1813600B1C50294ED95023464A4749F4
:101CF0001078DBB2FF2202284BD10868444C454DD6
:101D0000267890432A78964254D9227824782E78DF
:101D1000023B5D10A31B6B435201D31A10335B11BE
:101D20001843086001F070FF031F012B45D83A4BA0
:101D30001B78002B06D0394B1B78002B02D00020DB
:101D400002F01AF9A122364B92009978354B4A439A
:101D50001B689B18832292009B181B78033B012B66
:101D600003D8AF20400002F03FF901222E4BDA8267
:101D700070BD237824785BB264B2FF33FF341B0458
:101D800024021B190138ABE7CAB2022AAED20223E1
:101D9000ACE70868254C264D267890432A78964271
:101DA00008D9227824782D78023B5B10641B6343AA
:101DB0005201B2E72378DBB2B2E70228D5D11D4B3E
:101DC0001B78013B022B03D91B4B1B78022BCCD178
:101DD0006C20C8E79809FF1FFC0FFF1F3C64FF1F22
:101DE000FF3F0000141003404064FF1F0C1003402D
:101DF00000100340D50BFF1F7211FF1FB4000340FA
:101E00008C09FF1F680AFF1F490AFF1F9400034047
:101E1000460AFF1F470AFF1FF908FF1F2209FF1F7D
:101E2000300DFF1F3409FF1FBC0BFF1F440AFF1FAB
:101E3000450AFF1F1C09FF1F2309FF1F10B502F0F1
:101E400033F80022014B1A8010BDC0463A64FF1FD0
:101E500010B502F041F8A121054A89009478054A9D
:101E600061431268044B5218528C1A8010BDC04650
:101E7000300DFF1F3409FF1F3A64FF1F10B50D4BD3
:101E80000D4A9978A1239B004B431268D218531D29
:101E9000D97F0A4B1B88994209D2441C07D0C82815
:101EA00005D0D2695B1A5A43054B5343C01801F061
:101EB0000BFF10BD300DFF1F3409FF1F3A64FF1FD9
:101EC0007102000070B5244D2B68002B28D001F062
:101ED00033FF2B68D8402B680400002B27D001F07B
:101EE00053FE2B68D8401D4B1D4A9978A1239B00B7
:101EF0004B431268D118D25C91239B00002A20D05A
:101F0000CA580132CA50174B17491B6808688342E8
:101F100014D3D23B181A012A1AD0144B186070BD82
:101F200001F00AFF124B196801F026FED3E701F019
:101F30002BFE0F4B196801F01FFED4E70D495B180B
:101F4000E8E7CA500C4B1B68DB68E418201AE4E78A
:101F5000F530FF30E1E7C0461C08FF1F300DFF1FC2
:101F60003409FF1F9C09FF1F3C64FF1FA009FF1FCE
:101F70001808FF1F2DFF3F004464FF1F70B50400C9
:101F80000D00282916D10300A433C2881B889B1A90
:101F90000B4A9BB293420DD906006A3605223100E6
:101FA000653001F051FF002804D13100200001F01C
:101FB0004BFE70BD2900200001F0C6FEF9E7C046C7
:101FC000FE7F0000F8B50500012001F095FF134CDD
:101FD000A36AA26A9342FBD1114E336001F08CFEDA
:101FE0001049030008601048426894460F4A176879
:101FF0000022BC4501D24268BA1A0D48026032681C
:10200000AD18A422E562606A520302436262094A83
:102010001278002A01D00F3B0B60F8BD00F00040A1
:10202000340AFF1FE408FF1F28100040180AFF1F92
:102030001C0AFF1F1C09FF1F70B580241025E40532
:10204000A3682B43A36001F0C7FEA368AB43A36062
:1020500070BD0000F7B5160080221C001023D205C9
:102060000191916805000B43936000225A4BD730D1
:102070001A6001F079FD9D232A002F009B00EB5888
:10208000CA3201210092FC37002B01D00021009AB6
:10209000386801F0E1FD2900009BCB311A784F4BE5
:1020A000D3351A604B780A781B0213438A781204DE
:1020B0001A43CB781B061343494A1BBA13604B796A
:1020C0000A791B0213438A7912041A43CB7931002F
:1020D0001B061343434A1BBA13606B782A781B0212
:1020E0001343AA7812041A43EB781B0613433E4AA3
:1020F0001BBA1360019A330213433C4A13603C4BF2
:1021000022001B1B9C4603293DDCB3089A001300E8
:102110005142B21A032A46D1354AE018511A827840
:102120004078120400020243E05C043302430A6078
:102130000022FF2B4BDDF0222E4B12011A600F22E2
:102140002D4B1A602D4A1368002BFCD00023224A25
:1021500027491360091B321D0B191B68043A180A22
:1021600023706070180C1B0EA070E3700434002AFA
:10217000F2DC802210213B68D20501333B6093687A
:102180008B439360F7BD6346D578981893782D06F6
:102190001B042B43157804392B43557804322D0248
:1021A0002B430360AFE7022A0AD1114AE05C511ABF
:1021B000E2185278120202430A6004339BB2B7E776
:1021C000012AB5D10A4A521AE15C1160F5E70849C3
:1021D00059180A600433ACE7000004403C00044096
:1021E0003800044034000440300004400C00044037
:1021F00000010440040004401000044014000440A6
:10220000F7B5150080221C001023D20500919168BB
:1022100007000B4393600023654AD730136001F039
:10222000A3FC9D233E009B00F9583B00CA363200B8
:10223000FC33002900D07FE0586801F00DFD390023
:1022400032785C4BCB311A604B780A781B0213430F
:102250008A78AC4612041A43CB78281D1B06134318
:10226000554A1BBA13604B790A791B0213438A79CA
:1022700012041A43CB791B061343504A1BBA13604E
:102280004B7A0A7A1B0213438A7A12041A43CB7AD6
:1022900021001B0613434A4A1BBA1360009A2B0203
:1022A0001343484A13602200474B1B1B0093009BBB
:1022B000CE785B1801938B7836061B0433430E7877
:1022C000043833434E78043136023343019E336081
:1022D0000328ECDC0321A808431C9B002940800054
:1022E00003292BD13849E5185E18A9786D78E35C8D
:1022F00009042D02294319433160030008330021EA
:10230000FF2B2DDD314B324919600F21314B196004
:10231000012327490B60304B19680029FCD00621A6
:102320001B680B40042B20D080220020D20593682C
:102330000A318B439360FEBD01217DE7022908D15C
:1023400021495D18E1184978E35C090219432960C5
:10235000D3E70129D3D11C495918E35C0B60CCE7C2
:102360001948181801600433CAE7002310490B60AC
:102370006346002B0CDC3B00FC335A681021013211
:102380005A608022D205936801208B439360D2E784
:10239000009B9B181B68190A13705170190C1B0EB7
:1023A000D37004235B4291709C440432E0E7C04642
:1023B000000004403C000440380004403400044065
:1023C000300004400C0004400001044004000440BC
:1023D000080F0000100004401400044070B5061EF1
:1023E00019D002225A4B9B799343012B13D1594B9D
:1023F0001A78FF2A0FD15A78FF2A0CD19A78FF2A2F
:1024000009D1DA78FF2A06D11A79FF2A03D15B793C
:10241000FF2B00D199E0504B0C201A78012A08D0EC
:1024200000224E4D1A7029780B00093B042B01D86D
:10243000212070BD4B1F012BFAD9454CA37B042BE7
:1024400000D982E0A279032A00D97EE09A1ED2B296
:10245000012A02D860881F2877D9002E56D0012E75
:1024600073D1A0880128E3D0002907D1581E032882
:1024700003D801F055FB121715122E702978481E4B
:10248000032811D80025364B1D602823237501F041
:10249000B3FBA84227D0A580CAE702212970EDE747
:1024A0000421FBE70321F9E707390129C0D82D49A9
:1024B0000968C96A8906BBD52B4908780028B7D1B5
:1024C000012A01D9002BB3D102230B708021274DA3
:1024D000263389012878237501F016FC802128789D
:1024E000890101F019FC0123A380214B1B78002BEB
:1024F0000AD0FA2280211F4B92001B8809025A43FE
:102500001A4B187801F088FD002092E701F08CFD4D
:102510002B78A680073B012B03D917482E7001F0BA
:10252000C3FB114B114C1A78002A06D080210022DF
:10253000207889011A7001F0E7FB01F095FB8021FA
:102540002078090201F0E0FBDEE7122071E7C046C7
:10255000A60BFF1F6B09FF1F1A09FF1F1C09FF1F96
:102560004809FF1F4464FF1F2309FF1F1B09FF1FAA
:102570002109FF1F2C09FF1F0010004010B5002982
:1025800001D001F079FB10BDF7B5604B019199784E
:10259000A1239B004B435E4A060014681022E418F6
:1025A000D6235B00E0583623FF33E35C00279343D8
:1025B000222B41D1574B0F3A1A600760012501F0D9
:1025C00003FC019B1880E8235B00E35C002B01D037
:1025D000B34258DD0023504FFB70AD33FF33E35857
:1025E0001A68002A03D09B88DB439B071DD0382341
:1025F000FF33E35C002B18D09B235B00E35C002BD4
:1026000013D1D133FF33E35CB3420EDAA4235B0072
:10261000E15AE018090A023101F08EFC2300012280
:10262000FE33013E01351A87FA70E8235B00E35C54
:10263000002B2AD0A8B2FEBD03683D00002BBED0FF
:1026400081880430090A023101F076FCD6235B0050
:10265000E3581F60B2E72300B133BA00FF33985844
:10266000013781880430090A023101F065FCE82352
:102670005B00E35CBB42EEDCE822F61AED180023B7
:102680005200A354A6E70027F1E7200001F04CFB1D
:1026900000281FD0002E1DDD7319882647190193CD
:1026A000B600200001F018FB5A3080002018406866
:1026B000013581880430090A023101F03DFC200017
:1026C00001F04AFBA3590133A351BD4202D0019B43
:1026D0009D42E6D1114BE35C002BABD095239B00D0
:1026E000E35C002BA6D00E4BE15A0029A2D00D4A84
:1026F000A35C994202D90133A3549BE700231A211A
:102700002000A35401F058FB94E7C046300DFF1F92
:102710003409FF1F00140340E010FF1F5A0200009D
:10272000720200005E0200000D4970B54A6E0D4C49
:10273000D2038B69D20BA24206D80B4D0224AA42C7
:1027400004D901F041FC70BD02246442E218150076
:102750007E2425402242F4D0A3432B438B61F0E733
:1027600000F000400A200000FC1C0000F8B51D4BE2
:102770001D4F1A78002A10D1BA7B002A02D10132EB
:102780001A7003E0032AFAD0022AF8D001F034FAD2
:1027900000220120154B1A70F8BD154B154D1C6811
:1027A000154B9E7801232B702878C0B200F09EFB59
:1027B000BB7B002B0BD101F017FAA1239B007343C5
:1027C000E41883239B00E41823782B70E4E7032BA1
:1027D00002D101F019FBF0E70020022BDCD101F05F
:1027E000B3F9EAE71C09FF1FA60BFF1F2309FF1F10
:1027F0003409FF1F490AFF1F300DFF1FF0B587B0D6
:102800000EAD2F780FAD2D780593AC4663461400BE
:102810000E4D0CAA12782E7803930D9B0092019313
:102820002200059B029701F0E7FA2E70012C01D0DF
:10283000042C08D1802206498B889343054A1278DC
:10284000D20113438B8007B0F0BDC0461C09FF1FA7
:102850006C11FF1F7809FF1F0B001B3B70B50400B4
:102860003020E02B0DD81300E025493BFF3B9BB205
:10287000ED00AB4205D8034B200019825A8201F0CB
:1028800083FA70BD8410FF1F10B501F08DFB054B5E
:1028900000205B68052B04D9034A5268D20200D499
:1028A000980810BD00100040FCE100E070B501F098
:1028B000BBFB0D4B1B68FC33DC691D6AFFF7E4FFB3
:1028C0006419844204D2094B01241B68002B07D0F1
:1028D00004220024064B1A70064A9369013393615F
:1028E00001F0C2F9200070BD4464FF1F9809FF1F6A
:1028F0002309FF1FFC0FFF1F70B50C4D2B68FC3325
:102900005C6A01F091FBFFF7BFFF2B680025FC33E9
:102910009B6AE318834204D2054B1B68AB4200D18B
:10292000051B01F0A1F9280070BDC0464464FF1FDB
:102930009809FF1FD722044B92009B5810B5002B1B
:1029400000D0984710BDC0460000FF1F10B501F031
:10295000CFF8FFF7EFFF2749274BCA6D274C1A40E6
:1029600084235B001343CB65254B1B68186A01F079
:10297000C3FA244B244A1A60244B254A1A60A02229
:10298000244B52001A60244B187801F0BDFA200045
:10299000224901F001FA0023A3600233A360204B17
:1029A0002049236003232048A36001F0F5F9102299
:1029B0001E4BFF201A60802252031A60802292036D
:1029C0001A60802212041A6001F0D6FA012001F088
:1029D0008BF9FA20400001F047FA582001F004FB7F
:1029E000134801F019F9012001F0E6F8072001F081
:1029F0009BFA10BD00F0004000FEFEFF14100040E6
:102A00004464FF1F000003400180063DBC000340FA
:102A100034080000A40003404A0AFF1F71020000AE
:102A2000C3090000FFFF3F002810004000E100E064
:102A300030750000674E336888331B6883F308885D
:102A400001F01AFA644A6549136800200B401360CC
:102A5000634B644A1B68934200D1A6E001F0BCF8C6
:102A60000221614A13688B431360FFF76FFF5F4BCE
:102A70005F4C1878C0B201F0BFFA0023A3600233A4
:102A8000A3605C4B0120236001F036FA0323A360AE
:102A900001F012FA040001F087FA050001F00CFAC7
:102AA000554B186001F0B8F9544B1968621A531E5F
:102AB000A14200D213008022D203934201D39B0291
:102AC0009B0A3268D16AC90700D471E04C491C0CDA
:102AD00009689BB24C4359432402090A641803262F
:102AE0004849FC3293680A6847489B1A474A076876
:102AF000126847499B18474A9A1833409208DB19D5
:102B00000A600360042B03D9013233400A6003607A
:102B10000E684149A619300001F02EF83F4F3E499A
:102B20003B68C3183B603000019301F095F93C4EBF
:102B30003068081838493060884205D9019B013354
:102B40003B6001F089F9316001F076FA354B1B7872
:102B5000002B0DD001F028FA334B621B19681218B4
:102B60008A4232D24919091B091A304801F014F976
:102B70002F4E337A002B0ED001F016FA621BF1684B
:102B80001218914224D94919091B091A294801F040
:102B900003F900233372284B83F3088801F0ECF823
:102BA000002001F019F801F00FF801F015F85CE7CA
:102BB000DC0199000234641A5900641A09214B435C
:102BC0008033CB40A408E41889E7FA218900CCE7D8
:102BD0001A49DBE74464FF1F1CF00040FFFFC1FF00
:102BE0000C0AFF1FB641210310000040490AFF1FD5
:102BF00014100040C3090000100AFF1F340AFF1F11
:102C0000380AFF1F200AFF1F280AFF1F1C0AFF1F88
:102C1000240AFF1FC4090000710200006008FF1FA2
:102C20002C0AFF1F1C09FF1FE408FF1F00100040B3
:102C3000740BFF1F3C10004000000020DC0500006A
:102C4000A022054B92009B5810B5002B01D098474D
:102C500010BD01F0C1F9FBE70000FF1FA122054BE9
:102C600092009B5810B5002B01D0984710BD01F081
:102C7000B3F9FBE70000FF1FA222054B92009B580F
:102C800010B5002B01D0984710BD01F0A5F9FBE766
:102C90000000FF1FA322054B92009B5810B5002B8C
:102CA00001D0984710BD01F097F9FBE70000FF1F26
:102CB000A422054B92009B5810B5002B01D09847D9
:102CC00010BD01F089F9FBE70000FF1F70B501F0AE
:102CD0006BF94F4B186001F067F80400C30702D48A
:102CE00001F0DAF870BD00224A4B1A604A4B18789E
:102CF0000138042829D800F013FF0320181C2400F1
:102D0000200000F051FF0128ECD0444C2378042B24
:102D10006ED101F0E9F80028E4D001F03DF9582027
:102D200001F062F902232370DCE7200001F044F98E
:102D3000E9E7200001F018F8E5E7200001F024F9A8
:102D4000E1E7200001F0C0F8DDE700F05DFF0500DD
:102D5000012808D1324B1B78053B012B03D82000FA
:102D6000FFF76EFFD1E72D4B1B78022B01D0052B0F
:102D700020D1022D28D12B4B9B7BAB431CD12000B3
:102D8000FFF76CFF264B18780128BED16405BCD430
:102D9000244925224B7B034205D1233A13405A4252
:102DA000534126331A000B7D9342AED9322001F0F5
:102DB000D3F8AAE7022D07D1194B1B78052B11D1A7
:102DC0002000FFF759FFDDE7012D0BD1012B03D1C7
:102DD0002000FFF75FFF98E7062B03D12000FFF7E5
:102DE00067FF92E7200001F0F7F8022D8DD1C9E7C7
:102DF000032B04D10C4B987C00F0F6FF72E7072BF5
:102E000000D06FE7094B987B00F03EFF6AE7C046B1
:102E10009C09FF1F9809FF1F9009FF1F2309FF1F2F
:102E20001C09FF1FA60BFF1FBC0BFF1FD40BFF1FAE
:102E3000FA210A4B0A4A49001A640A4A5A500A4AB5
:102E400004395A50094A08319A64094A5A50094AC1
:102E50005C315A50084ADA667047C0460000FF1FCE
:102E6000FD27FF1FF928FF1FAD28FF1FDD23FF1FD0
:102E70006D27FF1F7D1EFF1F511EFF1FF7B50B0C97
:102E8000FF270122009300233C001E001D009446F2
:102E9000019089B262469A401000084018413618E5
:102EA000B6B2FF2F02D1012E00D19FB2009802408E
:102EB0001A41AD18ADB2FF2C02D1012D00D19CB248
:102EC0000133102BE6D10320012E07D1012D04D1AF
:102ED000019B2401E4191C700138FEBD102EFCD1A9
:102EE0000238102DF9D00230F7E700008023F7B543
:102EF0009C46264B264F01932649274A274D284CAE
:102F0000284B02281AD1604638600868264E3040A7
:102F1000802636033043086001990978002909D1D9
:102F20001660224A2A60224A2260E02219689143F0
:102F3000A03A1BE08021C9021160F2E766463E60BC
:102F40000F68194E3E408027FF023E430E600199F4
:102F5000097800290DD1176001280ED1154A2A6081
:102F6000154A2260E02219689143C03A0A431A6068
:102F7000F7BD802189021160EEE7E0210F4A02438C
:102F80002A600F4A22601A688A43F0E74B0AFF1F43
:102F9000E0000340D80003409000034000000340DD
:102FA0005000034040000340FFFFE3FF0280063D66
:102FB000804508220180063D806608220080069830
:102FC00080550822F8B51E4B80261A680020140090
:102FD0003440324232D11A681A4F32431A60012209
:102FE0003B68063093433B6000F086FF0122164D9C
:102FF0002B681E432E603B680A2613433B608027E4
:10300000BF00124B1B683B4211D1013EF6B2FF2EAE
:1030100009D17E220E4B1C682B68E40B14409343AD
:1030200023432B6005E0082000F066FFE9E7002E4F
:10303000EFD180222B68600893432B60F8BDC04617
:10304000C4F000405CF0004018F0004068F0004020
:1030500060F0004010B500F0E7FE01215820034A5F
:1030600000F082FFFFF7AEFF10BDC046600AFF1FF1
:1030700010B578220021034800F0C6FF00F064FF7D
:10308000002010BD3867FF1F70B5040000F0CCFFB2
:1030900000230C200B4A010059438D18515C002974
:1030A0000DD0A14208D1012300246B7000F004FE72
:1030B00000F0DAFD200070BD01330A2BEBD11224A1
:1030C000F6E7C0463867FF1F70B5040000F0ACFF9C
:1030D000002319001D000D4A1078002806D0A042D8
:1030E0000CD1557001310C320A29F5D1002B0AD1CF
:1030F00000F02AFF00F0B8FD002070BD5078461E99
:10310000B0411B18EEE700F0D7FDF3E73867FF1F6B
:10311000F7B504000C20002384460E4D019267464B
:103120005F43E85D7E19A04212D000280BD10A4B04
:103130009C4662461B7808331370019B70707C5567
:103140007160B360FEBD01330A2BE8D10320F9E7BB
:103150000720F7E73867FF1F3467FF1F8020F8B5A7
:10316000484BC0051B68C1248360474BFF251A6884
:10317000012313434361454BA4001A68444B40218B
:103180001A60444B1A68444B1A60444B1A59AA43BC
:103190001A51C52292009E58AE4331438026995061
:1031A0009F583F49F6010F403E439E509E5880274E
:1031B0003602360A3043985080201A5900020A40DD
:1031C00002431A5104341A59364E3F0432408026C5
:1031D0003A431A511A5936061202120A32431A5148
:1031E00008341A5980260A4002431A51C322920019
:1031F0009F58B446AF4337439F509F58294E0F40C6
:1032000007439F509F583740802636043743802617
:103210009F509F5836063F023F0A37439F50C022B7
:103220001F59AF433A431A511A591202120A164350
:10323000C6221E5192009C58AC4365462C439C50BC
:103240009C5800250C4020439850C72080001A58F5
:10325000154C1140C02212020A431A50134B1B781E
:10326000DB08AB4201DC0020F8BD2378002B06D040
:10327000A368002B00D0984701350C34EEE71220EC
:10328000F2E7C0464443FF1F4043FF1FB0F0004039
:103290003067FF1FB4F000402C67FF1F00E100E023
:1032A000FF00FFFFFFFF00FF3867FF1F3467FF1FAE
:1032B000030010B51F2809D8072200201340072457
:1032C00004490A78A24313430B7010BD0023062063
:1032D000F5E7C0463467FF1F054B06491B780A68AF
:1032E00005485B0702401B0B134300200B6070472F
:1032F0003467FF1F1CF00040FFFFC1FF70B50C25B5
:10330000FFF7EAFF0A4B1C780A4BE4086543ED1807
:10331000002C01D1200070BD2B78002B06D06B68EB
:10332000002B00D09847013C0C3DF1E71220F2E75A
:103330003467FF1F2C67FF1F1FB5002102220B00FF
:1033400001910091052000F0A7FC02230B490A68B7
:103350001A42FCD120230393039B5A1E0392002B95
:10336000FAD1074A1368002BFCDA0B246C442000C6
:10337000012100F061FC207804B010BD90C800402D
:1033800000C8004013B504000A4B0193019B002BB9
:1033900001D1112016BDFFF7CFFF230003400442E7
:1033A00005D0052000F0A8FD019B013BEDE71800CA
:1033B000F0E7C046FFFFFF0707B500F035FE8022AB
:1033C0000821D205936A0191002B01D1073991623E
:1033D00002210C4A11600199481E01900029FAD17E
:1033E00003311160053101910199481E01900029B6
:1033F000FAD11160002B02D18022D205936200F035
:1034000033FC07BD00C00040F0B52D4C89B02378D7
:10341000002B4FD1FEF7D2FA02232A4F03903A68CD
:103420001A42FCD120230693069B5A1E0692002BBB
:10343000FAD1254E3368002BFCDA0120FFF7A2FFFA
:10344000011E02D0112009B0F0BD0300032201903B
:10345000009005AD9F2000F01FFC0321280000F024
:10346000EBFB02233A681A42FCD120230793079B07
:103470005A1E0792002BFAD13368002BFCDA012088
:10348000FFF780FF0028DDD10398FEF7ABFAAA789A
:103490006B7811041B020B4329780B436360130004
:1034A000113B0A49052B07D801239340A3600B6009
:1034B000012323700020C6E780231B03F6E7C046E4
:1034C0002C43FF1F90C8004000C800409808FF1F11
:1034D0001E4B30B55A6818781D4B85B0D318594229
:1034E0004B4101210093002300F09EFB194B1A4A27
:1034F00002259A6300221A6510325A658022C4217F
:103500009D65164B1648D202DA6789004258154B62
:1035100080241A4080231B0413434350642341201A
:103520000393E40500F006FA402000F003FA656218
:10353000039D6B1E0393002DFAD103236362FFF7F3
:103540003BFFA562FFF760FF05B030BD3843FF1FAA
:1035500095FFFEF700C80040050001FF04E100E010
:1035600000E100E0FFFF00FFF0B585B00700FEF7C7
:1035700025FA022305002D4C22681A42FCD1202393
:103580000093009B5A1E0092002BFAD1284E3368FC
:10359000002BFCDA0120FFF7F5FE002803D01124F0
:1035A000200005B0F0BD234B2360022322681A429D
:1035B000FCD120230193019B5A1E0192002BFAD1CA
:1035C0003368002BFCDA0120FFF7DCFE0028E6D18F
:1035D000194B1F60022322681A42FCD12023029358
:1035E000029B5A1E0292002BFAD13368002BFCDAA0
:1035F0000120FFF7C7FE0028D1D1104B2360022322
:1036000022681A42FCD120230393039B5A1E039283
:10361000002BFAD13368002BFCDA0120FFF7B2FE51
:10362000041EBCD12800FEF7DDF9B9E790C80040C0
:1036300000C8004001000006A8C800400180000149
:1036400010B50020FFF790FF10BD000010B5064B2D
:1036500018705960FFF73CFF00211320034AFFF761
:1036600057FD002010BDC0463843FF1FD134FF1F57
:10367000F0B5040085B003920291FEF79FF988220D
:1036800063035B0B52051A438023DB059D6A80238D
:10369000274F0092BA68002601901B039A420CD96A
:1036A000F82326001B041E401C4206D08022214B1A
:1036B00052025E6219680A431A60002D0BD100F0B5
:1036C000B3FC02221C4B1A608023DB055A62013ACC
:1036D0009A6200F0C9FA0023039A934220D1002D88
:1036E0000AD100F0A1FC144B03221D608023DB05EE
:1036F0005A629D6200F0B8FA8023BA681B039A42AE
:1037000008D9002E06D000220A4B0C495A621A68CA
:103710000A401A600198FEF765F9002005B0F0BD77
:10372000009A0299D2181278CA540133D4E7C046DD
:103730002C43FF1F00C8004000C00040FFFFFEFFF9
:10374000F0B587B0029103920400FEF737F90190BB
:1037500000F06AFC802302250122234EDB05356040
:103760005D629A6200F080FA204F3B682B42FCD1E8
:1037700020230493049B5A1E0492002BFAD11C4D63
:103780002B68002BFCDA0120FFF7FCFD002802D09B
:10379000112007B0F0BD2000039A029900F0BCFB95
:1037A000022304003A681A42FCD120230593059BAA
:1037B0005A1E0592002BFAD12B68002BFCDA01204F
:1037C000FFF7E0FD051EE3D100F02EFC802303226D
:1037D000DB0535605A629D6200F046FA0198FEF7FB
:1037E00001F9E0B2D5E7C04600C0004090C80040F3
:1037F00000C80040F0B5802489B00600FEF7DEF86E
:10380000E405A36A02250393029000F00DFC012356
:10381000304F3D606562A36200F026FA2E4C2368AB
:103820002B42FCD120230593059B5A1E0592002BA9
:10383000FAD12A4D2B68002BFCDA0120FFF7A2FDFC
:10384000002803D01124200009B0F0BD244B2360D0
:10385000022322681A42FCD120230693069B5A1E9B
:103860000692002BFAD12B68002BFCDA0120FFF71F
:1038700089FD021EE6D11B4B03211E60030001904F
:103880000090202000F008FA022322681A42FCD19E
:1038900020230793079B5A1E0792002BFAD12B680F
:1038A000002BFCDA0320FFF76DFD041ECAD100F0E7
:1038B000BBFB80230322DB053C605A629C6200F064
:1038C000D3F9039B002B01D1FFF776FD0298FEF799
:1038D00089F8B8E700C0004090C8004000C8004028
:1038E0000100000694C8004007B5000201910422BF
:1038F000000A01A9FFF724FF0EBD000073B5050003
:1039000005240B4AA3005B429B1819686B46DE1D19
:103910003000FFF7B3FA022804D133782B55013C6D
:10392000EFD276BD052CFCD00128FAD10230F8E7A1
:10393000140900111F2807D8012380228340D205D3
:1039400091680B43936070473F2808D80123802279
:1039500020388340D20551690B435361F3E75F2858
:10396000F1D80123802240388340D205116A0B43ED
:103970001362E8E71F2807D8012280218240C90589
:103980008B6893438B6070473F2808D801228021C1
:1039900020388240C9054B6993434B61F3E75F28A8
:1039A000F1D80122802140388240C9050B6A934337
:1039B0000B62E8E71F2810D880230200DB05153AC8
:1039C0001968012A06D820229143196019680A4310
:1039D0001A60704701228240F6E73F2811D8802301
:1039E0000200DB05353AD968032A06D81022914334
:1039F000D960D9680A43DA60EBE7012220388240B7
:103A0000F5E75F28E5D842238022181A413B83401E
:103A1000D205516A99435162516A0B435362D8E708
:103A200010B50400012813D1A022184992050B6893
:103A30005B015B0913430B60154B164A1968114073
:103A4000154A0A431A60402219680A431A6010BDD9
:103A50000028FCD101000A2000F016FA21000B20FA
:103A600000F012FAC0220A4B920019680A43402162
:103A70001A601A688A431A60B022044912060B6859
:103A80005B015B0913430B60E1E7C04614F00040A3
:103A90001CF000407F00FEFF80FD010072B6074A67
:103AA0001368013313600422054B1A600023054A92
:103AB00013608022D2055360FEE7C0467808FF1FDE
:103AC000C0F00040C4F0004005490B68002B05D150
:103AD000044A0A6004490A60044A13607047C046F9
:103AE000140AFF1F841E0000380AFF1FC4F00040A4
:103AF0000023034A1360034A1360034A13607047AC
:103B000054F0004040F1004044F1004002B47146DE
:103B100049084900095649008E4402BC7047C04616
:103B200002B4714649084900095C49008E4402BC50
:103B30007047C04603B47146490840004900095A1D
:103B400049008E4403BC704701B40248844601BC5E
:103B5000604700BF19FA000001B40248844601BC66
:103B6000604700BFE927000001B40248844601BC59
:103B7000604700BF8944000001B40248844601BC8C
:103B8000604700BF090E000001B40248844601BC32
:103B9000604700BF6D0B010001B40248844601BCC0
:103BA000604700BFE94C010001B40248844601BCF3
:103BB000604700BF0134010001B40248844601BCE3
:103BC000604700BFE512010001B40248844601BC11
:103BD000604700BF8552010001B40248844601BC21
:103BE000604700BF016C010001B40248844601BC7B
:103BF000604700BFE9F6000001B40248844601BCFA
:103C0000604700BFA9D8000001B40248844601BC47
:103C1000604700BFDD0C010001B40248844601BCCE
:103C2000604700BF8D11010001B40248844601BC09
:103C3000604700BFC56D010001B40248844601BC65
:103C4000604700BF3D71010001B40248844601BCD9
:103C5000604700BF85C1000001B40248844601BC32
:103C6000604700BF2144000001B40248844601BC03
:103C7000604700BF9DA9000001B40248844601BC12
:103C8000604700BFE9D4000001B40248844601BC8B
:103C9000604700BFC1F7000001B40248844601BC80
:103CA000604700BF496D010001B40248844601BC71
:103CB000604700BFC1A5000001B40248844601BCB2
:103CC000604700BF21A9000001B40248844601BC3E
:103CD000604700BF8937010001B40248844601BC37
:103CE000604700BFD9B0000001B40248844601BC5F
:103CF000604700BF6911010001B40248844601BC5D
:103D0000604700BFBD5C010001B40248844601BCAD
:103D1000604700BFB352010001B40248844601BCB1
:103D2000604700BF0D52010001B40248844601BC47
:103D3000604700BF71B0000001B40248844601BC76
:103D4000604700BFE90B010001B40248844601BC92
:103D5000604700BF51B8000001B40248844601BC6E
:103D6000604700BF5976010001B40248844601BC97
:103D7000604700BF0534010001B40248844601BC1D
:103D8000604700BF7997000001B40248844601BC37
:103D9000604700BF116E000001B40248844601BCB8
:103DA000604700BF2D6C010001B40248844601BC8D
:103DB000604700BFBD0B010001B40248844601BC4E
:103DC000604700BF53B9000001B40248844601BCFB
:103DD000604700BFCD0C010001B40248844601BC1D
:103DE000604700BFDD3F000001B40248844601BCCB
:103DF000604700BF4DF9000001B40248844601BC91
:103E0000604700BF9D6A000001B40248844601BCBF
:103E1000604700BF75F8000001B40248844601BC49
:103E2000604700BFC166010001B40248844601BC7E
:103E3000604700BFED68010001B40248844601BC40
:103E4000604700BFDDB5001101B40248844601BCE3
:103E5000604700BFCD4C010001B40248844601BC5C
:103E6000604700BF090E000001B40248844601BC4F
:103E7000604700BF8512010001B40248844601BCBE
:103E8000604700BFC9A9000001B40248844601BCD4
:103E9000604700BF59A2001101B40248844601BC2A
:103EA000604700BFDD0A010001B40248844601BC3E
:103EB000604700BF8D82000001B40248844601BC07
:103EC000604700BF156B010001B40248844601BC85
:103ED000604700BFF935010001B40248844601BCC7
:103EE000604700BFF9ED000001B40248844601BC00
:103EF000604700BF01D7000001B40248844601BCFE
:103F0000604700BF0189000001B40248844601BC3B
:103F1000604700BFEDA5000001B40248844601BC23
:103F2000604700BF9573010001B40248844601BC9C
:103F3000604700BFF90D010001B40248844601BC8E
:103F4000604700BFC115010001B40248844601BCAE
:103F5000604700BFADAE000001B40248844601BC1A
:103F6000604700BF6137010001B40248844601BCCC
:103F7000604700BF0167010001B40248844601BCEC
:103F8000604700BFED6B010001B40248844601BCEC
:103F9000604700BFF535010001B40248844601BC0A
:103FA000604700BF6DF6000001B40248844601BCC2
:103FB000604700BFC95C010001B40248844601BCEF
:103FC000604700BF0934010001B40248844601BCC7
:103FD000604700BFD1AE000001B40248844601BC76
:103FE000604700BFE917010001B40248844601BCE4
:103FF000604700BF7912010001B40248844601BC49
:10400000604700BF8914010001B40248844601BC26
:10401000604700BFB70E000001B40248844601BCEF
:10402000604700BF8B52010001B40248844601BCC6
:10403000604700BF75A9000001B40248844601BC76
:08404000604700BFD5440100F8
:10404800020000008ABE00110100000090BC0011AF
:104058000200000086BE0011010000008840FF1F1A
:104068000200000098BC001101000000C061FF1FA1
:104078000200000084BE0011030000003461FF1F2D
:1040880012000000020000008ABE001101000000BA
:10409800D8BC00110200000086BE0011010000001B
:1040A800D5BC001102000000E2BC001103000000B2
:1040B8006F61FF1F0200000084BE001103000000B2
:1040C8008461FF1F0200000086BE0011010000008D
:1040D800D4BC001102000000E0BC00110300000085
:1040E8004561FF1F0200000084BE001103000000AC
:1040F8006661FF1F020000008ABE00110100000077
:1041080018BD00110200000086BE00110100000069
:10411800D141FF1F020000002ABD0011010000006C
:1041280013BD00110200000086BE0011010000004E
:10413800D041FF1F0200000028BD0011010000004F
:104148008C61FF1F0200000086BE00110100000004
:10415800CF41FF1F0200000026BD00110100000032
:1041680003BD00110200000086BE0011010000001E
:10417800CE41FF1F0200000024BD00110100000015
:10418800FEBC00110200000086BE00110100000004
:10419800CD41FF1F0200000022BD001101000000F8
:1041A800F9BC00110200000086BE001101000000E9
:1041B800CC41FF1F0200000020BD001101000000DB
:1041C800F4BC00110202020202020000000000001A
:1041D8000D0C0000B14B0011774B001178BD001198
:1041E80090011D0018001800FFFF070102030405D5
:1041F80006020106000000000000000000000000A8
:1042080000000000000000000000000000000000A6
:1042180003000000020000008ABE00110100000037
:1042280098BD00110200000086BE001101000000C8
:104238008C42FF1F02000000A2BD00110100000017
:10424800BA61FF1F0200000084BE001103000000D5
:104258002464FF1F0200000086BE00110100000058
:104268008C42FF1F02000000A0BD001101000000E9
:10427800BC61FF1F0200000084BE001103000000A3
:104288001C64FF1F126C6C6C00000000005800409A
:10429800151600000001000000000111FFFF0000DA
:1042A8005048593600000000000000000B000500CF
:1042B800F0000000B4000028002800283075A00095
:1042C800A000A000A00000080008E001F000100015
:1042D8001000100010001000100050005000500096
:1042E80010001000D0070000000000000F000100BF
:1042F8000500307507001000010081FF0000000074
:10430800FF0000004174001149720011D96F0011BB
:10431800FFFF0100FF0000005D9E0011D99B001106
:10432800F19A0011000000000000000000000800E1
:10433800040000003B0001085902E0018821280020
:10434800FF000000020000008ABE0011010000000A
:1043580050BF00110200000086BE001101000000DD
:10436800C943FF1F0200000082BE001101000000C7
:10437800F067FF1F0200000086BE00110100000068
:10438800C843FF1F0200000080BE001101000000AA
:10439800C643FF1F0200000086BE00110100000096
:1043A800C443FF1F020000007EBE00110100000090
:1043B800BC43FF1F180018001D00900102000003F5
:1043C80002020000020000008ABE00110100000085
:1043D80064BF00110200000086BE00110100000049
:1043E8000C44FF1F020000007CBE0011000000000A
:1043F800000000000200000084BE0011030000005D
:064408001068FF1F20FFF9
:040000051FFF184180
:00000001FF
